:020000040000FA
:10000000805E0020E5000000B9320000D900000049
:1000100000000000000000000000000000000000E0
:10002000000000000000000000000000F1000000DF
:100030000000000000000000F3000000F5000000D8
:10004000F7000000F700000035380000F70000005E
:1000500065120000F7000000F7000000F700000044
:10006000F7000000F7000000F7000000F7000000B4
:10007000F7000000F7000000F7000000F7000000A4
:10008000F7000000F700000000000000F70000008B
:10009000B92D000075150000F7000000F700000002
:1000A0000D120000F7000000F7000000D911000059
:1000B000F7000000F7000000D91E0000F700000064
:1000C0000448854600F0D4FC004800478D550000E8
:1000D000C046C046805E00207046694604F0E0FEDF
:1000E000FFF7FEFF0448804704480047FEE7FEE7AD
:1000F000FEE7FEE7FEE7FEE7893E0000C1000000E4
:1001000030B50B46014600202022012409E00D46AF
:10011000D5409D4205D31D469540491B2546954037
:1001200040191546521E002DF1DC30BD70B500247B
:100130002546002801DA01244042002901DA012580
:100140004942FFF7DDFFAC4200D04042002C00D016
:10015000494270BDF0B51FB40646002082B0054686
:100160004024019100901BE0019922460F46304641
:1001700000F0BAFB049A059B801A994110D31046EF
:100180001946224600F0A0FB361A8F4101972246FD
:1001900001200021009F00F097FB38184D4100908E
:1001A0002046641E0028DFDC019B00982946324669
:1001B00007B0F0BD0549064A08685043054A801853
:1001C00008604008704701490860704740020020FD
:1001D0006D4EC6413930000003460B439B0703D0E8
:1001E00009E008C9121F08C0042AFAD203E00B78FC
:1001F0000370401C491C521EF9D27047D2B201E074
:100200000270401C491EFBD270470022F6E710B571
:1002100013460A4604461946FFF7F0FF204610BD74
:100220000321001D401E037812021A43491EF9D50E
:1002300010467047034603220870000A491C521EEC
:10024000FAD51846704770B504460D46072310705E
:100250000E06000A3043090A521C5B1EF7D52046E1
:10026000294670BDF8B502464A40D40F42004B0003
:1002700052085B089A4202D20246084611464A00DA
:1002800023D0C30D4A00DDB2120EAD1A202D35DA8F
:1002900049020126490AF6058A19002C00D052426B
:1002A00020214F1B1146B9402A411018C20D9A4215
:1002B00021D0002C17D0012D08DCDA05801AD20FCE
:1002C0008019D207DBB200F03BFBF8BDDA05801ADB
:1002D000012340001B06C01880185A428018CA0F1C
:1002E0001043490007E04908C2071143DA05801AA4
:1002F00080194008801800F01BFBF8BD6100012246
:10030000511A001BF7E70122D2075140AAE7012248
:10031000D2075040A6E7024670B54A40D30FDB072C
:1003200040002DD04A002AD0010E140E0002120205
:100330000919400A520A8418E50104465443000A88
:10034000120A2E045043A4194219200CC543AA18BE
:10035000120C0125AD03521C521912047F392404DA
:1003600000D0521C104301D44000491EC2B20C06FA
:10037000C0092018401C4008802A02D003E0002059
:1003800070BD40084000002900DA0020184370BD0D
:1003900070B502464A40D50F40004A00ED074008BC
:1003A0005208002814D0002A12D0C40DD30D4102E7
:1003B0000120C0055202490A520AE41A091812180B
:1003C0007D34914201D3641C00E04900002C01DA25
:1003D000002070BD0023914201D3891A03434008D5
:1003E00049000028F7D100290AD0914202D1012109
:1003F000C90705E0914201D2012101E00121C94371
:10040000E005C018401900F093FA70BDF0B507463A
:100410000846584087B0C00F049048000E46590067
:1004200040084908BC1A884105D2384631461E4664
:1004300017460B4602465800400810434DD0300D79
:10044000039040055900400D490D0590401A029057
:10045000402873DA18030121000B090508430190B5
:1004600004980092002806D01146019A49420020C3
:10047000904100910190029840210A1A0199009838
:1004800000F022FA05460C466B4607CB00F03DFA19
:10049000C0197141039A0E0D0023D71756401A4612
:1004A0007A40164344D0049A002A2DD0029A012A99
:1004B000039A15DC1205C01A914101263605001C6D
:1004C0007141D20F059ED2070093019202962A46EF
:1004D000234600F07BFA07B0F0BD38463146FAE714
:1004E0001605234A0F46B218C01AB7410121090563
:1004F000001C4F4100187F41114618187941E20F46
:1005000010436D19644113E0E2076D081543640858
:10051000C2071443039A01261205C01A91413605F9
:10052000001C7141CE07400830434908C0185141B2
:100530002A46234600F03DFACDE7FFE70498012262
:100540004000C117121A00238B4104983146C4178A
:10055000381AA141EEE730B40124E407634030BC0F
:1005600054E730B40124E407614030BC4EE700009A
:100570000000E0FFF0B51FB488B00B990998002483
:1005800048400999C00F490049080991C0070B99D3
:100590000090490049080B9109990898A64608431C
:1005A0001CD00B990A98084318D0099801244000E0
:1005B000420D4800410D099824050003000B20431B
:1005C00009900B980003000B20430B9050181C4916
:1005D0004018002201901446104605E00020014614
:1005E0000DB0F0BD032801DA034600E003239C466A
:1005F000C11A0AAE0AE05F0008ADED5B4F00F75B81
:100600007D430027AA187C41491C5B1E6145F2DD31
:10061000410004AB5A522104120C0A43240C401C22
:100620000828DFDB01980290009970460191009044
:10063000059B049A0799069800F0C8F9D0E70000D6
:100640000DFCFFFFF0B50C465C4085B0E40FE407FD
:1006500003944C0000266408590094464908024659
:100660000296224321D062460A431ED06200570DF3
:100670004A000E032303550D012402462C4924058C
:10068000781B1B0B360B4018234326436146009012
:100690001C46501AB44103D30098401C009002E05D
:1006A000921800985B41002803DA0020014605B04B
:1006B000F0BD0020012109050746864611E0644689
:1006C0001D46141BB54106D36546521BB341744603
:1006D00007430C43A646CD07400849082843921813
:1006E0005B4105460D43EAD11046184313D06046DE
:1006F000194650407140084306D06046101AB34175
:1007000006D20122002306E000220123DB0702E0DB
:100710000122D2435310009874460105381C6141F0
:10072000029C039D0019694100F043F9BFE70000F6
:10073000FD03000010B500229623114600F000F9D9
:1007400010BD00000EB5C217C10F5040CA074018B7
:100750000021054B0293019200910A460B4600F0DE
:1007600035F903B000BD0000330400000EB50549A3
:100770000291002100910A460B46019100F026F9F2
:1007800003B000BD33040000C20F4100400201234A
:10079000400ADB05D207090EC0187F2901DA0020C4
:1007A0007047962903DC9623591AC84001E0963910
:1007B0008840002AF4D040427047000070B5CD0F49
:1007C0004A0009030123090B1B0519430B4BED07D5
:1007D0000024520D9A4201DA002070BD074B3433D9
:1007E0009A4203DC9A1A00F07FF802E0044951189B
:1007F00088402C43F1D0404270BD0000FF03000050
:10080000CDFBFFFFC20FD207400040080BD0C10D47
:100810000723DB01C91840020905400A1143C20839
:1008200040071143704700200146704710B500296A
:1008300004DB0124E40740428C412146002B04DB09
:100840001C460123DB075242A3418B4200D1824266
:1008500010BD000010B5002904DB0124E40740426C
:100860008C412146002B04DB1C460123DB0752424E
:10087000A341994200D1904210BD0000CB0FDB078D
:10088000490010B5490802460A4307D00A0D07245B
:100890000903E401090B121B002A01DC002010BD32
:1008A000C900440F0C43C100E018D205801800F0C5
:1008B0003FF810BD0122D207002800DB101A0029E2
:1008C00000DB511A8142704710B5202A04DB014633
:1008D000203A9140002010BD914020239C1A0346ED
:1008E000E3401943904010BD10B5202A04DB0846B0
:1008F000203AD040002110BD0B46D340D0402024E8
:10090000A21A91400843194610BD10B5202A06DBF3
:10091000CB170846203A1041C1170B4306E00B469F
:100920001341D0402024A21A91400843194610BD1B
:10093000002904DA401C490001D1400840007047FA
:1009400070B40024050C05D11024000402D1002944
:1009500021D01124050E01D100020834050F01D168
:100960000001241D850F01D18000A41C002801DB9B
:100970004000641C002908D020252E1B0D46F540A0
:10098000A14000D001212943084301061B1B000A96
:10099000DB1D02D5002070BC7047DB0518188018DD
:1009A0000029F8DA401C4900F5D170BC400840002D
:1009B000704710B5002B08DA0024401C61419218E2
:1009C0005B411A4301D14008400010BDF0B51FB48F
:1009D00082B005460C0003D0084603F01DFE02E07D
:1009E00003F01AFE20300246009021462846FFF709
:1009F0006BFF049B059A04460F46184311430843B6
:100A000014D0184610431BD0009840210A1A1846EB
:100A10000599FFF769FF05460E46009A0599049867
:100A2000FFF752FF084305D0012004E02046394675
:100A300007B0F0BD0020C11705430E432C433743D8
:100A400000990E986305401A7905E40A00220C43C8
:100A5000FD0A0A3002D500200146E9E70105101918
:100A600069410C9C0D9D00196941FFF7A2FFDFE76A
:100A7000064C0125064E05E0E36807CC2B430C3CF1
:100A800098471034B442F7D3FFF71EFB886A000082
:100A9000A86A000070B58C180578401C6B075B0FC6
:100AA00001D10378401C2A1106D10278401C03E0D2
:100AB00006780E70401C491C5B1EF9D12B0705D42B
:100AC0000023521E0DD40B70491CFAE70378401C1A
:100AD000CB1A921C03E01D780D70491C5B1C521E42
:100AE000F9D5A142D8D3002070BD00000146064AC6
:100AF000106907231B0402469A4310461A460A400F
:100B00001043014A1061704700FA0140012806D1E4
:100B10000649096920221143044A116105E003498D
:100B2000096920229143014A1161704700FA01408E
:100B30000146054A1069000900010A07120F104317
:100B4000014A10617047000000FA0140012806D1F7
:100B50000649096840221143044A116005E003492F
:100B6000096840229143014A1160704700FA014030
:100B7000012806D10649096801221143044A11607F
:100B800005E00349096849084900014A11607047B6
:100B900000FA01400146064A1068082302469A43BB
:100BA000104608220A401043014A106070470000B6
:100BB00000FA01400146064A1068042302469A439F
:100BC000104604220A401043014A1060704700009A
:100BD00000FA0140012806D10649096802221143A2
:100BE000044A116005E00349096802229143014A61
:100BF0001160704700FA01400148806880B2704778
:100C000000FA014010B5012000F00EFB03F010FBCC
:100C1000012003F01FFB022003F0FAFA012003F089
:100C2000E5FA0420FFF784FF0120FFF76FFF04209F
:100C3000FFF7C0FF0120FFF7CDFF01208004FFF781
:100C400055FF0020FFF7A6FF044800F04DF80020F4
:100C5000FFF77CFF0020FFF78BFF10BDFF070000B0
:100C600010B5012000F0E0FA03F0E2FA012003F0F1
:100C7000F1FA022003F0CCFA012003F0B7FA0820C1
:100C8000FFF756FF0120FFF741FF0420FFF792FF17
:100C90000120FFF79FFF01208004FFF727FF0020BE
:100CA000FFF778FF044800F01FF80020FFF74EFF21
:100CB0000020FFF75DFF10BDFF0700000548C0687A
:100CC000FF2101310840002801D001207047002099
:100CD000FCE7000000FA0140FF2001300149C86034
:100CE0007047000000FA01404105490D014A51607A
:100CF0007047000000FA014010B5012000F094FA9E
:100D000003F096FA012003F0A5FA022003F080FA1E
:100D1000012003F06BFA0F20FFF70AFF0120FFF715
:100D2000F5FE0420FFF746FF0120FFF753FF0748B9
:100D3000FFF7DAFF01208004FFF7D8FE0020FFF75D
:100D400005FF0020FFF714FF10BD0000FF070000A3
:100D5000F8B505460E46002E22D02868002800D19E
:100D6000F8BD2C6801E0274664686068002802D05E
:100D70002088B042F7D12088B04210D109480078CD
:100D8000401E084908702868A04202D160682860A7
:100D900001E060687860204604F07CFB002400BF1E
:100DA00000BFDDE720000020F3B58DB00C46A2495E
:100DB000C878FFF7DBFC0546A04AA14BFFF7DAFB3A
:100DC0000B910A900D98FFF71DFD099108900B9B60
:100DD0000A9AFFF72BFD02D2012020755FE09649A9
:100DE000C878FFF7C3FC0546944A954BFFF7C2FB52
:100DF000924A944B07910690FFF708FB0B910A90DB
:100E00000D98FFF7FFFC099108900B9B0A9AFFF7DA
:100E10000DFD07D2207D012801D120753FE0022081
:100E200020753CE084498878FFF7A0FC0546834A9A
:100E3000834BFFF79FFB0B910A900D98FFF7E2FCA5
:100E4000099108900B9B0A9AFFF7F0FC02D202204E
:100E5000207524E078498878FFF788FC0546774AB2
:100E6000774BFFF787FB754A764B07910690FFF7A4
:100E7000CDFA0B910A900D98FFF7C4FC09910890E8
:100E80000B9B0A9AFFF7D2FC07D2207D022801D1E2
:100E9000207504E00020207501E000202075207DF1
:100EA000012802D10020E077C3E0207D022852D142
:100EB000614880786049C978884249DD5E4989780F
:100EC0005D4AD278881AFFF73DFC05465B4A5C4BC9
:100ED000FFF750FB0991089057498878FFF746FCC7
:100EE0000546564A564BFFF745FB039102900D9875
:100EF000FFF788FC01910090039B029AFFF72BFB00
:100F00000022514B05910490FFF734FB07910690A6
:100F1000099B089AFFF796FB0B910A90FFF7AEFC2E
:100F200007463846FFF76EFC05460022464BFFF7A2
:100F300091FC01D2454F05E000213846FFF7BAFC8D
:100F400000D200273846FFF71FFC40B2E07770E080
:100F50000020E0776DE038498878FFF707FC374AD2
:100F6000374B0B910A90FFF705FB05460522520708
:100F7000374BFFF75BFC5AD22F498878FFF7F6FB17
:100F800005462E4A2E4BFFF7F5FA05225207304B45
:100F900005910490FFF7E5FA0991089026498878B1
:100FA000FFF7E4FB0546254A254BFFF7E3FA0391DB
:100FB00002900D98FFF726FC01910090039B029A86
:100FC000FFF7C9FA0022234B05910490FFF7D2FAEC
:100FD00007910690099B089AFFF734FB0B910A9042
:100FE000FFF74CFC07463846FFF70CFC054600228D
:100FF000184BFFF72FFC01D2174F09E03846FFF7D7
:1010000001FC054600221346FFF710FC00D2002722
:101010003846FFF7F7FB054600220B4BFFF7F6F9C2
:101020000B910A90FFF7CAFB40B2E07701E0142071
:10103000E0770FB0F0BD0000ED0000209A9999997B
:101040009999B93F9999C93F000034400000A041E7
:1010500099991940000054400000A04210B50121A8
:10106000054800F05BF9022000F086F8002210210C
:10107000024802F05FF910BD07000001400D00407A
:101080007FB506460D4614466A462946304600F0AE
:10109000D9FE0098A84227D16846C079002823D1FC
:1010A000E007C00F002803D16846407900281BD113
:1010B000E007C00F002803D068464079012813D10B
:1010C00002202040002803D16846807900280BD1F7
:1010D00002202040002803D068468079012803D1EF
:1010E0006846007902281DD0029500206946C87321
:1010F000E007C00F002801D1487302E001206946D3
:10110000487302202040002802D16946887302E01B
:1011100001206946887302206946087302A9304697
:1011200000F0B8FF7FBD7FB505460C466A462146F4
:10113000284600F087FE0098A0420FD16846C0798B
:1011400000280BD168464079002807D1684680798D
:10115000002803D16846007903280BD002940021AF
:101160006846C173417381730321017302A9284644
:1011700000F090FF7FBD000070B5054600240026FA
:1011800000F046F8002802D1012000F04DF80024BC
:1011900016E00120A04006462846304000280ED028
:1011A0000C4800680121A14088430A4908600846AC
:1011B0008168620003209040014306488160641CFE
:1011C000042CE6D300F024F8012802D1002000F01E
:1011D0002BF870BD00FC014010B500F005F80028A8
:1011E00001D000F00DF810BD04480069C007C00F21
:1011F000002801D0012070470020FCE7006001407A
:1012000001200149086170470060014070470000FB
:10121000044800680007000F0A2801D10120704728
:101220000020FCE700E00140012803D10A21034A25
:10123000116002E00521014A1160704700E00140A1
:10124000012806D10649896901221143044A9161A6
:1012500005E00349896949084900014A91617047DD
:1012600000240040002070470548C069FF2101317B
:101270000840002801D0012070470020FCE7000052
:101280000024004010B50446012C02D11148036827
:1012900013E0022C03D10F484038C36B0DE0032C40
:1012A00003D10C484038836B07E0042C03D1094874
:1012B0004038436B01E007480368180CD94389B2F2
:1012C000884203D1D8B200F07FF802E06B2000F032
:1012D0007BF810BD40FBFF1F012806D10649096BB2
:1012E000C2071143044A116305E00349096B490031
:1012F0004908014A11637047002400400146064A2C
:10130000106B130502469A4310461A460A401043D2
:10131000014A1063704700000024004030B50246C7
:101320000B4600200F2424061440FF252D066419C7
:10133000002C09D06419002C08D06419002C08D0A6
:101340006419002C0BD107E00D4809E00C48001D82
:1013500006E00B48083003E009480C3000E000BF0D
:1013600000BF00280BD092B201219140002B03D086
:1013700004680C43046002E004688C43046030BDE0
:10138000202400400146064A50680F231B040246F1
:101390009A4310461A460A401043014A506070476B
:1013A00000240040012806D1064949680122114362
:1013B000044A516005E00349496849084900014A67
:1013C00051607047002400400146044A9068000ABA
:1013D0000002CAB21043014A9060704700240040E6
:1013E00010B504462068FFF7CDFF2079FFF7DAFF3C
:1013F00010BD00000146064A106807231B02024682
:101400009A4310461A460A401043014A106070473A
:10141000002400400146064A106807231B040246C8
:101420009A4310461A460A401043014A106070471A
:1014300000240040012806D10749096842061143EB
:10144000054A116006E004490968012252069143E9
:10145000014A116070470000002400400146054A1F
:101460001068C008C0004A07520F1043014A1060BC
:10147000704700000024004010B504462068FFF7C4
:10148000EDFF6068FFF7B6FFA068FFF7C3FF207BA2
:10149000FFF7D0FF10BD0000012806D106494969B9
:1014A00001221143044A516105E003494969490891
:1014B0004900014A51617047002400400146064A34
:1014C000506907231B0202469A4310461A460A40F7
:1014D0001043014A5061704700240040F8B50446AB
:1014E0000F461D462E46422C05D10320A87200202F
:1014F000E872B07308E0522C06D100231422314662
:101500001831024803F020FCF8BD000072000020F2
:1015100070B50A460021002300BF12E001248C4070
:10152000234614461C40002C0AD0046801258D4037
:10153000AC430460C4684E000325B540AC43C460AE
:10154000491C1029EAD370BD032001218907486096
:10155000704700000146C800054BC21804231068FC
:101560001840002801D0012070470020FCE700004F
:101570000404004010B50720FFF7ECFF012807D155
:10158000072000F007F8012802D1072000F012F828
:1015900010BD000001460648806A012212048A40FC
:1015A0001040002801D0012070470020FCE7000017
:1015B00040040040012109048140014A91627047C2
:1015C00040040040F8B506460C46174600BF4021CF
:1015D000174800F0A2FD01218903154800F09FFD86
:1015E00000BF032002F0F2FB2102080E02F0EEFB26
:1015F0002104080E02F0EAFBE0B202F0E7FB00254E
:1016000005E0FF2002F0E2FB7055681C85B2BD4288
:10161000F7DB00BF4021064800F081FD012189036E
:10162000034800F07CFD00BF00F090F8F8BD00001A
:10163000800C0040F7B584B07D21490106988842AE
:1016400002DD002007B0F0BD049802900020039056
:10165000059C069D002D0CD0200A461C3002001B64
:10166000A84201D32F4601E03002071B012003905E
:1016700001E00020039061E000BF4021324800F00B
:101680004CFD01218903304800F049FD00BF0620D0
:1016900002F09CFB00BF40212B4800F040FD0121DF
:1016A0008903294800F03BFD00BF00BF40212648C8
:1016B00000F033FD01218903234800F030FD00BF15
:1016C000022002F083FB2102080E02F07FFB2104BE
:1016D000080E02F07BFBE0B202F078FB00200190E4
:1016E00009E002990878491C029102F06FFB019809
:1016F000401C80B201900198B842F2D300BF402153
:10170000114800F00CFD012189030F4800F007FD8E
:1017100000BFE419ED1B002D0CD0200A461C30023E
:10172000001BA84201D32F4601E03002071B012015
:10173000039001E00020039000F008F803980028CF
:101740009AD100BF7EE70000800C004010B500BFBA
:1017500000F006F8C007C00F0028F9D110BD000046
:1017600010B50A2003F006FD00BF40210E4800F02E
:10177000D4FC012189030C4800F0D1FC00BF0520F6
:1017800002F024FBFF2002F021FB044600BF4021B1
:10179000054800F0C4FC01218903034800F0BFFCA8
:1017A00000BF204610BD0000800C0040FFB581B096
:1017B00004460F463946204603F0CAFF002801D1EF
:1017C00005B0F0BDE41C6846407C012821D1617859
:1017D0006846017021784170E1788170A178C1700C
:1017E0000098FEF7C3FF0546244AFEF72CFD6179F9
:1017F0006846017021794170E1798170A179C170E9
:101800000098FEF7B3FF05461C4A083AFEF71BFD99
:1018100031E06846407C022814D1617817483230A4
:1018200001712178001D4170E1788170A178C1704B
:101830006179001F017021794170E1798170A1798E
:10184000C17018E06846407C032814D161780B48C9
:101850001230017721781C304170E1788170A178D5
:10186000C17061791C380176217918304170E179B5
:101870008170A179C1700120A2E700002A0E00202A
:1018800010B501210448FFF749FD0022202103483B
:1018900001F069F910BD000007000001400D004093
:1018A0000146054A1068800880008A07920F10439D
:1018B000014A1060704700000010004010B500227F
:1018C00001210903014801F04EF910BD800C0040D0
:1018D000F7B503460D460021002207E00126964099
:1018E0002E40002E01D0114602E0521C102AF5D3E2
:1018F00000BF102A00D1FEBD314FDE1BBB4211D00C
:1019000008DC304E9E19002E09D0402E08D0802EC3
:1019100051D106E0402E06D0802E4CD104E000BF0D
:1019200000BF00BF00BF00BF254E4036B34203D00A
:10193000234E8036B34202D10B2903D93CE00F2954
:1019400000D939E0032901D800200CE0042903D391
:10195000072901D8012006E0082903D30B2901D863
:10196000022000E00320164E803EB34200D1001D4D
:10197000134E403EB34200D10830114EB34200D165
:101980000C300F4E4036B34200D110300C4E803632
:10199000B34200D114300C4E3469029E012E02D1A4
:1019A0008640344304E0012686402746B7433C4640
:1019B000054E346100E000BF00BF00BF9BE70000A0
:1019C000C00C004000F4FFBFC00D0040F0B502465F
:1019D0000D4600230027002407E00120A0402840F6
:1019E000002801D0234602E0641C102CF5D300BF70
:1019F000102C01D13846F0BD2E4E901BB24211D0B2
:101A000008DC2D481018002809D0402808D080286C
:101A10004CD106E0402806D0802847D104E000BF22
:101A200000BF00BF00BF00BF22484030824203D049
:101A300020488030824202D10B2B03D937E00F2B94
:101A400000D934E0032B01D800210CE0042B03D390
:101A5000072B01D8012106E0082B03D30B2B01D85B
:101A6000022100E0032113488038824200D1091D81
:101A700010484038824200D108310E48824200D1DD
:101A80000C310C484030824200D11031094880307E
:101A9000824200D114310948406901268E4030400D
:101AA00001268E40B04200D1012700E000BF00BFF8
:101AB0003846A0E7C00C004000F4FFBFC00D004056
:101AC000F0B502460C460021002307E001269E40A7
:101AD0002640002E01D0194602E05B1C102BF5D3E6
:101AE00000BF102B00D1F0BD2D4FD61BBA4211D034
:101AF00008DC2C4E9619002E09D0402E08D0802EDE
:101B000049D106E0402E06D0802E44D104E000BF2B
:101B100000BF00BF00BF00BF214E4036B24203D01D
:101B20001F4E8036B24202D10B2903D934E00F296F
:101B300000D931E0032901D800200CE0042903D3A7
:101B4000072901D8012006E0082903D30B2901D871
:101B5000022000E00320124E803EB24200D1001D60
:101B60000F4E403EB24200D108300D4EB24200D17D
:101B70000C300B4E4036B24200D11030084E803649
:101B8000B24200D11430084E7569012686403540B6
:101B9000054E756100E000BF00BF00BFA3E7000075
:101BA000C00C004000F4FFBFC00D0040F8B5054672
:101BB0000E4617461C4603223146284600F022F8FE
:101BC0003146284600F0A4F8224631462846FFF761
:101BD0007FFE3A463146284600F014F8C82003F04C
:101BE000C9FA31462846FFF76BFF1E20002805DBA7
:101BF000C206D20E01219140014A116000BFF8BD1A
:101C000080E200E0F7B5034615460021002408E015
:101C10000126A640019F3E40002E01D0214602E051
:101C2000641C102CF4D300BF102C00D1FEBD354F26
:101C3000DE1BBB4211D008DC334E9E19002E09D0AA
:101C4000402E08D0802E58D106E0402E34D0802E71
:101C500053D132E000BF00BF00BF0F2900D94DE0D3
:101C6000032901D800200CE0042903D3072901D857
:101C7000022006E0082903D30B2901D8042000E044
:101C80000620204E803EB34200D108301D4E403E1B
:101C9000B34200D110301B4EB34200D118301B4E5E
:101CA000B268032686401746B7433A462E4686401A
:101CB0003243164EB26021E000BF0B2900D91DE06F
:101CC000032901D8002006E0042903D3072901D8FD
:101CD000022000E004200B4E8036B34200D10830D1
:101CE0000A4EF268032686401746B7433A462E4608
:101CF00086403243054EF26000BF00BF00BF00BF08
:101D000094E70000C00C004000F4FFBFC00D00408D
:101D1000F0B502460D460020002407E00126A6404B
:101D20002E40002E01D0204602E0641C102CF5D37A
:101D300000BF102C00D1F0BD3F4FD61BBA4234D0AB
:101D400008DC3E4E9619002E2CD0402E2BD0802E33
:101D50006ED129E0402E02D0802E69D100E000BF74
:101D60000B2800D965E0032801D8002106E00428EB
:101D700003D3072801D8022100E004212E4E80362B
:101D8000B24200D108318007800F2D4E73680326C0
:101D90008E401F46B7433B4606468E403343284E8F
:101DA000736046E000BF00BF00BF234EC03EB2429A
:101DB00007D0214E803EB24203D01F4E403EB24279
:101DC00002D10F2800D934E01B4EB24202D10B28B9
:101DD00000D92EE0032801D800210CE0042803D309
:101DE000072801D8022106E0082803D30B2801D8D0
:101DF000042100E00621104E803EB24200D108319D
:101E00000D4E403EB24200D110310B4EB24200D1D5
:101E100018318007800F0A4E336803268E401F4614
:101E2000B7433B4606468E403343054E336000E0E1
:101E300000BF00BF00BF7EE7C00C004000F4FFBF42
:101E4000C00D0040F0B504460025002307E0012640
:101E50009E400E403546002D00D002E05B1C102B4A
:101E6000F5D300BF102B36D21D46116026680E40F8
:101E70003046E840012802D10126D67101E0002653
:101E8000D67166680E40EE403046012801D1967149
:101E900001E000269671A6680E40EE40304601280B
:101EA00001D1567101E000265671E6686F00FE40D0
:101EB000B007800F002802D1002616710BE0012820
:101EC00002D10126167106E0022802D102261671FF
:101ED00001E003261671F0BD10B501F0A9FF402105
:101EE0006548FFF773FD012823D140216248FFF7C1
:101EF000E7FD0120614908706148C08800280AD0C8
:101F00005F48C088401E81B25D48C180002902D16F
:101F100001205B4908715A484088002809D0584878
:101F20004088401E80B256494880002801D10120D7
:101F30000870202150484030FFF748FD012818D193
:101F400020214D484030FFF7BBFD20214A4840305A
:101F500000F0D9F800280CD140214748403000F06B
:101F6000D2F8002805D0012109034348803000F051
:101F7000CAF80121090340488030FFF727FD0128F6
:101F80000AD101033C488030FFF79AFD0121090383
:101F90003948803000F0B7F8402137484030FFF72B
:101FA00015FD012819D1402133484030FFF788FD45
:101FB00040213148403000F0A6F800280DD1012121
:101FC00009032D48803000F09EF8002805D101203B
:101FD0002C49087002202C490870082126484038F6
:101FE000FFF7F4FC012804D1082123484038FFF70B
:101FF00067FD0121490220484030FFF7E7FC012836
:1020000009D141021C484030FFF75AFD02F04CFA5A
:1020100001201E4908700121490217484030FFF78E
:10202000D5FC012809D1410213484030FFF748FD93
:1020300002F03AFA02201549087001210E48FFF714
:10204000C5FC012806D101210B48FFF739FD01200D
:102050000F49C8700121C90207488030FFF7B6FC5C
:10206000012807D1C10204488030FFF729FD012073
:102070000749087110BD0000C00C0040000000209E
:10208000020000201800002019000020B6000020E7
:1020900044000020F0B502460B4600210024002534
:1020A00000BF2DE001268E4034461E68264035468E
:1020B000A54224D110680646A6433046DE798E40FC
:1020C0003043106050680646A64330469E798E40E5
:1020D0003043506090680646A64330465E798E4095
:1020E000304390604F000326BE403446D068064619
:1020F000A64330461E794F00BE403043D060491C95
:102100001029CFD3F0BD02460020D3690B40002B2D
:1021100001D0012000E000207047816170474161DB
:1021200070470000F8B504460526E84840780028C6
:1021300011D1E648C07800280DD1E4484079002844
:1021400009D1E3480088052808DAE1480088401CE6
:10215000DF49088002E00020DD490880DD48C078C2
:1021600017280AD1DB480079392806D1D9484079A7
:10217000392802D1012020706070D64800793928B2
:1021800005D1D44840793A2801D10120A070E078E7
:10219000012822D10020E0700121CF48FFF7B3FFD2
:1021A00000281AD100BFCD4800794007C00F002891
:1021B00012D1CB49097904229143091DC84A1171F2
:1021C0004907C90F8900042211400846C34909790B
:1021D00091430143C14A117100BF2079012824D1E4
:1021E000002020710121C902BB488030FFF78BFF1E
:1021F00000281AD100BFB94800798006C00F002816
:1022000012D1B7490979202291432031B44A117182
:102210008906C90F4901202211400846AF490979B2
:1022200091430143AD4A117100BF2078002808D0C6
:102230000020207000F056FAA0602146A06800F04F
:102240009FFE607800280CD0A1480088052808DB94
:102250000120607000F09EF9206121462069FEF7A0
:10226000A3FDA078012804D10020A07000F084FA1A
:10227000A0619A4840788007C00F002802D1994891
:1022800000F050FE97480830FDF7CAFF0546954814
:10229000001DFDF7C5FF854202D30020607716E0E0
:1022A0009048001DFDF7BCFF00908E48001DFDF713
:1022B000B7FF07468B480830FDF7B2FF381A642194
:1022C000484305460099FDF71BFF40B26077207B2D
:1022D000012820D100BF814800798007C00F002865
:1022E00006D17E48007902218843801C7B49087111
:1022F00000BF00BF79480079C007C00F002806D191
:102300007648007940084000401C7449087100BFBD
:102310000020A07778E0207B022823D100BF6F48FF
:1023200000798007C00F002809D06C48007902218D
:1023300088436A49087111216B48FEF709FD00BF07
:1023400000BF66480079C007C00F002806D1634867
:10235000007940084000401C6049087100BFE07FE0
:10236000A07751E0607F642800D102E01D20205654
:10237000401C40B2A0771E202056142820DA00BF4F
:10238000564800798007C00F002809D053480079CB
:10239000022188435149087111215348FEF7D8FCA6
:1023A00000BF00BF4D480079C007C00F002806D10C
:1023B0004A48007940084000401C4849087123E021
:1023C00000BF464800798007C00F002809D0434865
:1023D0000079022188434149087111214248FEF7E2
:1023E000B7FC00BF00BF3D480079C007C00F002800
:1023F00009D03A4800794008400038490871102156
:102400003948FEF7A5FC00BFFFF73AFA2021324811
:102410008030FFF778FE002829D1002121200155C6
:1024200020200157052904DA005D401C41B220201C
:10243000015520200157052946DB284840788007B0
:10244000C00F002840D108212348C030FFF767FEA5
:1024500000BF224840788007C00F002806D11F48DF
:10246000407802218843801C1C4948702CE00021E0
:102470002020015521200157052904DA005D401C68
:1024800041B2212001552120015705291CDB1348A9
:1024900040788007C00F002816D008210E48C030B1
:1024A000FFF73BFE00BF0D4840788007C00F0028B3
:1024B00009D00A4840780221884308494870002121
:1024C0000948FEF745FC00BFF8BD000012000020DF
:1024D0006A00002030000020C00C004050020020A4
:1024E00066020020ED0000201C00002000B501461F
:1024F0000B0002F0A8F8091A0C0E11141706080AAE
:102500001A00692000BD9B20FCE79B20FAE79B2076
:10251000F8E7FF201E30F5E7FF20BE30F2E7FF208E
:10252000EB30EFE74120C000ECE74120C000E9E7D5
:1025300070B5002400250120FEF71AFBFEF7CCFB46
:1025400002F062FB002803D1FEF756FB054601E0CE
:10255000002070BD284602F0D3FA04462046F8E772
:1025600038B50020009000240120FEF701FBFEF7A3
:10257000B3FB02F049FB002803D1FEF73DFB044604
:1025800001E0002038BD204602F00CFB00900098CE
:10259000F8E70000F0B587B00026FEF75FFDFEF714
:1025A0005FFB10211C48FFF7BAFD052002F0BAFDC1
:1025B000132003F097F8041E27D008216170002132
:1025C000A17008202070204600F0EEF8074638463B
:1025D000FEF7B0F80190FEF715F9104A104B039181
:1025E0000290FDF7C7FF05910490FEF747F90546F5
:1025F0000C492846FDF78FFE064610210648FFF7D6
:102600008CFD204602F046FF00240020FEF7B0FAC1
:10261000304607B0F0BD0000400D0040FCA9F1D2EB
:102620004D62503FC3F548401FB50446072202A93A
:10263000002001F081F86846817B0170417B417088
:10264000017B8170817AC170417A0171017A417197
:102650000199009801F04AFC012814D16846007ADB
:1026600060716846407A20716846807AE0706846FA
:10267000007BA0706846407B60706846807B20705D
:10268000012004B010BD072202A9002001F054F877
:102690006846817B0170417B4170017B8170817A4A
:1026A000C170417A0171017A41710199009801F07C
:1026B0001DFC012813D16846007A60716846407A93
:1026C00020716846807AE0706846007BA07068469A
:1026D000407B60706846807B20700120D1E700203D
:1026E000CFE70000F0B587B0002600F0A3FDFEF7AD
:1026F00089FA08211C48FFF712FD052002F012FD9F
:10270000142002F0EFFF041E27D008216170002181
:10271000A17004202070204600F046F80746384695
:10272000FEF708F80190FEF76DF8104A104B039180
:102730000290FDF71FFF05910490FEF79FF80546F4
:102740000C492846FDF7E7FD064608210648FFF735
:10275000E4FC204602F09EFE00240020FEF708FA6A
:10276000304607B0F0BD0000400D0040FCA9F1D29A
:102770004D62503FD7A3004070B5FEF7BDFA13205D
:1027800002F0B0FF041E0AD0082161700021A17080
:10279000FFF7CEFE0546204602F07CFE0024002016
:1027A000FEF7E6F9284670BDFEB50446002000900D
:1027B000002509E0FFF7D4FE0746AA00E01C111827
:1027C0003846FDF737FD6D1CA1786278080210438A
:1027D000A842EFD800252EE06E1C25E0B200E11CD7
:1027E0005018FDF71DFD0746AA00E11C5018FDF723
:1027F00017FD874217D2B200E11C5018FDF710FDFB
:102800000190AA00E11C5018FDF70AFD0746B2002E
:10281000E01C11183846FDF70DFDAA00E01C111848
:102820000198FDF707FD761CA17862780802104335
:10283000B042D3D86D1CA178627808021043A84238
:10284000CAD8012002900BE002998A00E11C5018BE
:10285000FDF7E6FC0099401800900298401C029099
:10286000A178627808021043401E02998842EBD892
:10287000A278637810021843811E0098FDF740FC8F
:1028800000900098FEBD000010B501F04BFA042145
:102890000C48FFF742FC012002F06CFC04210948BF
:1028A000FFF73DFC042002F065FC04210548FFF71A
:1028B00034FC042002F05EFC04210248FFF72FFCE8
:1028C00010BD0000C00C004010B501F02BFA04212F
:1028D0000A48FFF724FC012002F04CFC04210748C1
:1028E000FFF71DFC042002F045FC04210348FFF71C
:1028F00014FC042002F03EFC10BD0000C00C00409F
:1029000070B504211348FFF70AFC01F0FBF980249D
:102910001BE004210F48FFF702FC012002F02AFC13
:1029200004210C48FFF7EFFB012803D12846204380
:10293000054602E02846A043054604210548FFF766
:10294000ECFB042002F016FC6410002CE1D12846B8
:1029500070BD0000C00C004010B501210648FEF714
:10296000DDFC00220421054800F0E4FC04210348BA
:10297000FFF7D3FB10BD000007000001C00C0040B2
:1029800070B5054601F0CEF980241BE020462840B2
:10299000002804D104211448FFF7BFFB03E0042101
:1029A0001148FFF7BCFB012002F0E4FB04210E48B4
:1029B000FFF7B5FB042002F0DDFB04210A48FFF716
:1029C000ACFB6410002CE1D1042002F0D3FB042105
:1029D0000548FFF7A4FB042002F0CCFB04210248C9
:1029E000FFF79BFB70BD0000C00C004010B5FFF767
:1029F000B3FF01F097F904210A48FFF790FB042187
:102A00000848FFF78CFB042002F0B4FB04210548C2
:102A1000FFF783FB042002F0ADFB04210148FFF720
:102A20007CFB10BDC00C004010B501F07BF9042107
:102A30000C48FFF772FB04210A48FFF76EFB0420E5
:102A400002F098FB04210748FFF769FB042002F01D
:102A500091FB04210348FFF762FB042002F08AFB8C
:102A600010BD0000C00C00400148024908607047DA
:102A70005A5A34120014014010B501210448FEF7DF
:102A80004DFC062003494860FFF7EEFF10BD000033
:102A900005000001001401401CB500200090012039
:102AA000694608716846FEF79BFC0120FEF7EAFBC9
:102AB0001CBD00000A20054908600548008CC0B212
:102AC0000449C861052001490860704700E00140E1
:102AD00000FBFF1F00F801401FB500240121194829
:102AE000FEF71CFC02211848FEF71DFB04211648C6
:102AF000FEF719FB0120FEF7CFFC07200002FEF7CE
:102B0000DDFC052002F00EFB0120FEF799FB05E03D
:102B100019200002844200D304E0641CFEF7A4FBE9
:102B20000028F5D000BF0120009000200190029005
:102B30000120694608736846FEF79EFC034802F0D0
:102B4000CDFA1FBD07000001400D0040001BB7007B
:102B500010B50020FEF7A4FEFFF79EFFFFF7AAFFC7
:102B6000FFF7BAFF10BD7FB506460D4614466A460C
:102B700029463046FFF766F90098A84217D1684603
:102B8000C079012813D16846407901280FD1002C63
:102B900003D168468079002809D1012C03D1684609
:102BA0008079012803D168460079002814D0029565
:102BB00001216846C1734173002C03D1002069468E
:102BC000887302E001206946887300206946087313
:102BD00002A93046FFF75EFA7FBD0000F8B5054652
:102BE0000E4600240027FEF713FB002802D1012027
:102BF000FEF71AFB002426E00120A04007462846E5
:102C0000384000281ED0002E07D11448406801210A
:102C1000A14088431149486006E0104840680121FE
:102C2000A14008430D4948600C48816862000320B8
:102C3000904081430948816000680121A140084318
:102C400006490860641C042CD6D3FEF7E1FA01287B
:102C500002D10020FEF7E8FAF8BD000000FC0140B8
:102C6000FFB587B015461E4600200490002D01D107
:102C70000BB0F0BD32780192D217130F019A9A1857
:102C800012110A235A433178CB171B0F5B181B1103
:102C90001B01CB1AD2183C235A4373780293DB17DB
:102CA0001F0F029BFB181B110A277B437078C71765
:102CB0003F0F3F183F113F01C71BDB19D21894B2D9
:102CC00006946A46D27F0192D217130F019A9A187E
:102CD00013110A2253436A46D17FCA17120F5218A2
:102CE000121112018A1A9B183C22534308AA127827
:102CF0000292D217170F029ABA1812110A277A43B2
:102D000008AF3878C7173F0F3F183F113F01C71B67
:102D1000D2199A1892B20592069C002D06D0294627
:102D20002D204001FDF702FA401C00E0012080B296
:102D3000039008A84078002816D1049010E0059868
:102D4000844201D1012093E7601984B22D20400113
:102D5000844201DB201A84B20498401C80B20490A3
:102D6000039904988842EADB002081E710B501222C
:102D700020210A48FFF7F7FE0122110307484030DF
:102D8000FFF7F1FE012240210448FFF7ECFE01228B
:102D9000082102488038FFF7E6FE10BD000D004014
:102DA00004488069C007C00F002801D00120704787
:102DB0000020FCE70034014010B500F009F80128BC
:102DC00005D1FFF7EDFF012801D100F00DF810BD8E
:102DD0000448406940210840002801D00120704784
:102DE0000020FCE700340140402001494861704761
:102DF0000034014010B501220649842000F05CF83F
:102E0000FF2101310448FFF788F980210248FFF7CC
:102E100084F910BD1A020020C00C004010B5012139
:102E20000B48FEF77BFA002280210A4800F082FA64
:102E30000022FF210131074800F07CFAFF21013117
:102E40000448FFF76AF980210248FFF766F910BDD0
:102E500007000001C00C004010B501220249842087
:102E600000F02AF810BD00001C02002010B5002060
:102E7000054908703022054900F037F83021034831
:102E8000FDF7C3F910BD00001D020020B30B0020A8
:102E900010B5FFF7C3FF80210548FFF740F9012077
:102EA00002F040F9FFF7D8FF01200249087010BD79
:102EB000C00C00401D020020F8B507460D4616461E
:102EC0000024FFF793FD7C20FFF75AFD3846FFF7FB
:102ED00057FD00BF04E0285DFFF752FD601CC4B23F
:102EE000B442F8DBFFF7A0FDF8BDF8B507460D4684
:102EF00016460024FFF77AFD7C20FFF741FD802075
:102F0000FFF73EFD3846FFF73BFD00BF04E0285DBC
:102F1000FFF736FD601CC4B2B442F8DBFFF784FD56
:102F2000F8BD000070B5044620460C30FDF778F976
:102F3000451C21460C312846FDF77CF920460C3013
:102F4000FDF76EF9E1210901884215D321460C31C4
:102F50000020FDF76FF920460830FDF761F90749B9
:102F6000884209D220460830FDF75AF9451C21460F
:102F700008312846FDF75EF970BD000030560100AB
:102F8000F3B58DB00C46A2494878FDF7EFFB054636
:102F9000A04AA14BFDF7EEFA0B910A900D98FDF7B0
:102FA00031FC099108900B9B0A9AFDF73FFC02D275
:102FB000012020735FE096494878FDF7D7FB05466E
:102FC000944A954BFDF7D6FA924A944B0791069096
:102FD000FDF71CFA0B910A900D98FDF713FC09916F
:102FE00008900B9B0A9AFDF721FC07D2207B012851
:102FF00001D120733FE0022020733CE0844908782F
:10300000FDF7B4FB0546834A834BFDF7B3FA0B91FA
:103010000A900D98FDF7F6FB099108900B9B0A9A10
:10302000FDF704FC02D20220207324E078490878DE
:10303000FDF79CFB0546774A774BFDF79BFA754AEF
:10304000764B07910690FDF7E1F90B910A900D98E8
:10305000FDF7D8FB099108900B9B0A9AFDF7E6FB58
:1030600007D2207B022801D1207304E000202073C6
:1030700001E000202073207B012802D1002020776E
:10308000C3E0207B022852D161480078604949782A
:10309000884249DD5E4909785D4A5278881AFDF711
:1030A00051FB05465B4A5C4BFDF764FA09910890B9
:1030B00057490878FDF75AFB0546564A564BFDF727
:1030C00059FA039102900D98FDF79CFB0191009035
:1030D000039B029AFDF73FFA0022514B05910490A1
:1030E000FDF748FA07910690099B089AFDF7AAFA9E
:1030F0000B910A90FDF7C2FB07463846FDF782FBAD
:1031000005460022464BFDF7A5FB01D2454F05E0E1
:1031100000213846FDF7CEFB00D200273846FDF7E8
:1031200033FB40B2207770E0002020776DE0384913
:103130000878FDF71BFB374A374B0B910A90FDF7D8
:1031400019FA054603229207374BFDF76FFB5AD257
:103150002F490878FDF70AFB05462E4A2E4BFDF74E
:1031600009FA03229207304B05910490FDF7F9F913
:103170000991089026490878FDF7F8FA0546254A8E
:10318000254BFDF7F7F9039102900D98FDF73AFBF7
:1031900001910090039B029AFDF7DDF90022234B79
:1031A00005910490FDF7E6F907910690099B089AAE
:1031B000FDF748FA0B910A90FDF760FB0746384689
:1031C000FDF720FB05460022184BFDF743FB01D21B
:1031D000174F09E03846FDF715FB05460022134658
:1031E000FDF724FB00D200273846FDF70BFB054610
:1031F00000220B4BFDF70AF90B910A90FDF7DEFA5E
:1032000040B2207701E0142020770FB0F0BD00001D
:10321000ED0000209A9999999999B93F9999C93FD8
:10322000000034400000A041CCCC1C4000005440C1
:103230000000A04210B501210648FEF76FF84021BA
:103240000548FDF770FF00220821034800F072F8DE
:1032500010BD000007000001400D004010B5002225
:1032600001218902044800F065F800220121890249
:10327000014800F05FF810BD000D004010B50022BD
:10328000012149020448FFF76EFC00220121490296
:103290000148FFF768FC10BD000D004010B501218A
:1032A00049020448FEF734F9012149020148FEF7BA
:1032B0002FF910BD000D00407047000010B5002828
:1032C00019DB1A4A03231B02D21883089B00D25829
:1032D0008307DC0EFF23A3409A438B071B0E840752
:1032E000E40EA3401A43114B032424021B19840843
:1032F000A4001A5118E00E4A03071B0F083B9B0855
:103300009B00D2588307DC0EFF23A3409A438B0710
:103310001B0E8407E40EA3401A43054B0407240F39
:10332000083CA408A4001A5110BD000000E100E010
:103330001CED00E07FB506460D4614466A46294658
:103340003046FEF77FFD0098A84217D16846C07945
:10335000002813D1002C03D16846407900280DD1F4
:10336000012C03D168464079012807D1684680794D
:10337000002803D168460079012813D00295002067
:103380006946C873002C01D1487302E001206946E8
:1033900048730021684681730121017302A93046F8
:1033A000FEF778FE7FBD0000FEB5FFF79BF9BC4934
:1033B0008860BC494878FDF7D9F90646BA4ABB4B44
:1033C000FDF7D8F804460D46B5498868FDF71AFAA6
:1033D00022462B4601910090FDF728FA1DD200BF2E
:1033E000B34800798007C00F002806D1B0480079A3
:1033F00002218843801CAE49087100BF00BFAC4861
:103400000079C007C00F002806D1A94800794008FC
:103410004000401CA64908715AE0A2490878FDF70F
:10342000A5F90646A04AA14BFDF7A4F804460D46AF
:103430009B498868FDF7E6F922462B4601910090EA
:10344000FDF7F4F920D200BF994800798007C00F3A
:10345000002809D0964800790221884394490871D0
:1034600011219448FDF774FC00BF00BF904800791B
:10347000C007C00F002806D18D48007940084000E1
:10348000401C8B49087123E000BF89480079800700
:10349000C00F002809D0864800790221884384495A
:1034A000087111218348FDF753FC00BF00BF80481D
:1034B0000079C007C00F002809D07D480079400876
:1034C00040007B49087110217A48FDF741FC00BF9C
:1034D000FFF760F8724908617249C878FDF746F94C
:1034E0000446714A714BFDF745F806460F466C4994
:1034F0000869FDF787F932463B4601910090FDF7D8
:1035000095F91DD200BF6A480079C006C00F002897
:1035100006D167480079102188431030644908714A
:1035200000BF00BF624800790007C00F002806D125
:103530005F4800790821884308305D4908715AE0E6
:1035400058498878FDF712F90446574A574BFDF75A
:1035500011F806460F4652490869FDF753F93246FD
:103560003B4601910090FDF761F920D200BF504821
:103570000079C006C00F002809D04D4800791021FD
:1035800088434B49087114214A48FDF7E1FB00BF0D
:1035900000BF474800790007C00F002806D1444803
:1035A00000790821884308304149087123E000BFB1
:1035B0003F480079C006C00F002809D03C48007978
:1035C000102188433A49087114213A48FDF7C0FB9D
:1035D00000BF00BF364800790007C00F002809D09F
:1035E0003348007908218843314908711321314853
:1035F000FDF7AEFB00BFFEF743F920212E48FEF792
:1036000082FD002833D10A2001F08CFD20212A48B8
:10361000FEF779FD002813D1082127484030FEF736
:103620007EFD00BF224840788007C00F002806D1E9
:103630001F48407802218843801C1D4948702DE0B6
:1036400008211D484030FEF768FD00BF184840784B
:103650008007C00F002809D0154840780221884310
:103660001349487000211348FDF772FB16E008214A
:1036700011484030FEF751FD00BF0D4840788007EB
:10368000C00F002809D00A48407802218843084921
:10369000487000210748FDF75BFB00BFFEBD00003E
:1036A00044000020ED0000209A9999999999B93F1A
:1036B000500200201C000020400D004010B50121E8
:1036C0001B48FDF72BFE002208211A48FFF732FEA7
:1036D0000022012117488038FFF745FA0022102107
:1036E0001448FFF727FE00210120C002FFF776FAF9
:1036F00010211048FEF711FD08210E48FEF70DFDC0
:10370000002204210B484030FFF714FE002208215C
:1037100008484030FFF70EFE042106484030FEF70F
:10372000FEFC082103484030FEF7F7FC10BD000006
:1037300007000001400D0040F8B507460D4616464B
:103740000024FFF753F96420FFF71AF93846FFF712
:1037500017F9FFF74BF96520FFF712F900BF06E0F4
:10376000FFF7CEF82855FFF78FF8601CC4B2701E23
:10377000A042F5DCFFF7C4F82855FFF7A5F8FFF7DE
:1037800053F9F8BDF8B507460D461646FFF72EF972
:103790006420FFF7F5F83846FFF7F2F8002404E05C
:1037A000285DFFF7EDF8601CC4B2B442F8DBFFF708
:1037B0003BF9F8BD0146064A5068062302469A4383
:1037C000104606220A401043014A5060704700002C
:1037D00000280040012806D106494968012211430A
:1037E000044A516005E00349496849084900014A13
:1037F0005160704700280040012806D10649096839
:1038000001221143044A116005E00349096849088F
:103810004900014A116070470028004010B5FFF7C9
:103820009BF8012240210248FFF79DF910BD0000DE
:10383000C00C00407047000070B50646FFF71EFD43
:10384000002E04DD652E02DA304601F06BFC01210A
:1038500049020E48FEF757FC0546012149020B4874
:10386000FEF751FC0446002D02D1012C00D170BDA1
:10387000012D03D1002C01D10220F8E7012D03D145
:10388000012C01D10520F2E70520F0E7000D0040F2
:10389000F0B58BB004460F463946204601F058FF7C
:1038A000002801D10BB0F0BDE41C002306226E49B4
:1038B000204601F049FA012304220AA9A01D01F0C3
:1038C00043FA0123022209A920460A3001F03CFAFA
:1038D0006846808CFCF74AFF644A654B0191009072
:1038E000FCF748FE039102900A98FCF73FFF05465B
:1038F000039B029AFCF78AFD5B4A0E320591049005
:10390000FCF7A1FC012304220AA920460C3001F097
:103910001BFA0123022209A92046103001F014FAF3
:103920006846808CFCF722FF504A514B0191009071
:10393000FCF720FE059104900A98FCF717FF03910D
:103940000290059B049AFCF761FD0546464A921DCC
:10395000FCF779FC0123042243493C312046123014
:1039600001F0F2F9012304223F4938312046163094
:1039700001F0EAF9012304223B49403120461A3084
:1039800001F0E2F9012304223749443120461E3078
:1039900001F0DAF9012304220AA92046223001F0BD
:1039A000D3F90123022209A92046263001F0CCF9DF
:1039B0006846808CFCF7DAFE2C4A2D4B0191009072
:1039C000FCF7D8FD039102900A98FCF7CFFE05465C
:1039D000039B029AFCF71AFD234A2E3205910490AC
:1039E000FCF731FC012304220AA92046283001F00B
:1039F000ABF90123022209A920462C3001F0A4F9D9
:103A00006846808CFCF7B2FE0546184A184BFCF756
:103A1000B1FD039102900A98FCF7A8FE0191009075
:103A2000039B029AFCF7F2FC0F4A263205910490A0
:103A3000FCF709FC012308220B491E3120464630C1
:103A400001F082F9012308220749163120464E3041
:103A500001F07AF90023082206A92046563001F029
:103A600073F901201EE700001C0E00207B14AE47F6
:103A7000E17A843F10B501213048FDF74FFC002268
:103A800080212F48FDF7FCFA0022FF2101312C484C
:103A9000FDF7F6FA0022012149022948FDF7F0FA64
:103AA00001212848FDF73AFC0021274800F06FF873
:103AB000FF210131244800F083F80021224800F062
:103AC0008CF80821204800F041F800211E4800F041
:103AD0006BF800211C4800F04EF800211A4800F055
:103AE00041F80021184800F0C3F80021164800F002
:103AF0009AF80021144800F07CF80021124800F0E8
:103B000085F80021104800F0A7F800210E4800F0C9
:103B1000BBF800210C4800F0C3F80B4800F0D2F8C5
:103B2000094800F0C9F8084800F0C9F8064800F054
:103B3000CCF80121044800F083F810BD0700000113
:103B4000800C004003000003004C014010B50A4601
:103B5000016838240B46A343194638231340194300
:103B6000016010BD0A46016849084900D307DB0F10
:103B700019430160704710B50A46016802240B46DC
:103B8000A3431946022313401943016010BD10B529
:103B90000A4601680124E4020B46A3431946234662
:103BA00013401943016010BD10B50A460168042492
:103BB0000B46A3431946042313401943016010BD6B
:103BC00010B50A460168FF2401340B46A343194689
:103BD000234613401943016010BD10B50A46016821
:103BE000C0240B46A3431946C02313401943016068
:103BF00010BD10B50A464168032464020B46A34376
:103C00001946234613401943416010BD10B50A46BA
:103C10004168FF2401340B46A34319462346134051
:103C20001943416010BD012904D14268CB021A43F7
:103C3000426004E042680123DB029A43426070471D
:103C4000012904D1426801231A43426003E042681B
:103C5000520852004260704710B50A46416820245D
:103C60000B46A3431946202313401943416010BD5E
:103C7000012904D1426802231A43426003E04268EA
:103C800002239A4342607047012904D142681023FD
:103C90001A43426003E0426810239A43426070472F
:103CA000012904D1426808231A43426003E04268B4
:103CB00008239A43426070470221816070470421C3
:103CC00081607047012181607047082181607047E1
:103CD00001460869C007C00F002801D001207047C5
:103CE0000020FCE70146086902221040002801D0AC
:103CF000012070470020FCE7014688697047416158
:103D00007047000010B501210448FDF707FB0022B1
:103D100004210348FEF727FF10BD00000700000143
:103D2000C00C004010B501210448FDF7F7FA00224D
:103D300004210348FFF7FEFA10BD00000700000150
:103D4000C00C0040FFB585B004460D4616460E9FD8
:103D500013A103C9049103906846047145718671EB
:103D6000C7710F99017269461098487202990198BB
:103D700000F0BCF8012810D1694610980873684615
:103D80000F99417387730899C173067445748474DD
:103D9000072203A90020FFF7F5FC09B0F0BD0000E1
:103DA00000000000010115001CB5002168460170EB
:103DB0004170022181700021C170402101710522F2
:103DC00069460B20FFF7DEFC1CBD000010B5044661
:103DD00021460A48FFF793FF00BF0848FFF782FF1C
:103DE0000028FAD000BF0548FFF772FF0028FAD07C
:103DF0000248FFF781FF0446E0B210BD004C0140CD
:103E000003B50A4840788007C00F002801D0012080
:103E10000CBD68464078012800D1F9E76846C078B3
:103E2000012800D1F4E70020F2E700005002002052
:103E30001FB500240120FDF72FFB07200002FDF72E
:103E40003DFB032001F06EF90120FDF7F9F905E0D3
:103E500019200002844200D304E0641CFDF704FA38
:103E60000028F5D000BF01200090002001900290B2
:103E70000120694608736846FDF7FEFA014801F023
:103E80002DF91FBD001BB7001920000302498860EF
:103E9000024803490860704700ED00E000127A0014
:103EA0003C02002010B572B6FEF7E6FD0D4801F0A9
:103EB00015F90A2001F036F9FEF74AFE0120FFF756
:103EC0009BFC0620FFF776FC0020FFF783FCFDF744
:103ED0003BFB01210448FDF721FAFEF7C5FD62B660
:103EE00010BD000000127A0007000001F3B582B097
:103EF0006E46337ADE17360FF61837110A267743E7
:103F00006E46307AC617360F361836113601861BC4
:103F1000BE19F2B26E46737ADE17360FF6183711F5
:103F20000A2677436E46707AC617360F3618361152
:103F30003601861BBE19F4B26E46B37ADE17360F11
:103F4000F61837110A2677436E46B07AC617360F31
:103F5000361836113601861BBE19F1B26E46F37A59
:103F6000DE17360FF61837110A2677436E46F07AB9
:103F7000C617360F361836113601861BBE19F5B234
:103F80006E46337BDE17360FF61837110A26774355
:103F90006E46307BC617360F361836113601861B33
:103FA000BE19F6B201966E46737BDE17360FF61811
:103FB00036110A277E436F46787BC7173F0F3F189D
:103FC0003F113F01C71BF619F6B20096632A11DCB8
:103FD000142A0FDB0C2C0DDC002C0BD01F2909DC64
:103FE000002907D0172D05DC01983B2802DC00983A
:103FF0003B2802DD002004B0F0BDA01E030000F04D
:1040000022FB0A0E1E061E071E1E081E091E00BFEA
:1040100000BF00BF1E2901DD0020ECE700BF9007B4
:10402000800F002803D01C2901DD0020E3E7900762
:10403000800F002802D11D2900DDDCE700E000BF71
:1040400000BF0120D7E701468868C007C00F0028DD
:1040500001D0012070470020FCE7F8B507460D4667
:10406000164600240BE0295D384600F00BF800BF2F
:104070003846FFF7E8FF0028FAD0601C84B2B4424B
:10408000F1DBF8BDCA05D20D42617047F8B50446B0
:104090000D460126E1781F488078814205D12179BB
:1040A0001C48801C4078814200D00226A0786428F9
:1040B00009D0A078012806D0A078022803D0A078E3
:1040C000032800D00026012E03D1E1210901124866
:1040D000C181FCF76FF807466421FCF727F80F024F
:1040E000FCF768F864210090FCF720F80F43B9B2A0
:1040F0000A480180E971090A29720120A87200208A
:10410000E872E87AA97A000208430B302E54304650
:10411000F8BD0000900000200200002012020020E4
:1041200010B50446204600F031F810BDF8B504463D
:104130000E4614480078012823D1217AE27908023A
:1041400010431149098888421BD1607B217B000202
:1041500008430006050C607B227B00021043FF220F
:10416000120210400012054327460E37012D06D1DA
:10417000607A33463A462946FDF7B0F900E000BFC1
:1041800000BFF8BD0E0200201202002070B50446E8
:1041900000BFE07AA17A000208430C3085B2E07AD1
:1041A000A17A000208430006010CE07AA27A00021C
:1041B0001043FF221202104000120143A172080AAC
:1041C000E0722A462146074801F0B8FF0646301241
:1041D0006055681C2654A81C82B221460248FFF78D
:1041E0003CFF70BDFFFF000000740140012806D1B4
:1041F0000649496A01221143044A516205E0034914
:10420000496A49084900014A5162704700F8014073
:104210000146064A506A0E2302469A4310460E2271
:104220000A401043014A50627047000000F8014004
:1042300000B507484368180CD94389B2884203D1B6
:10424000D8B200F019F802E01F2000F015F800BD08
:1042500040FBFF1F012806D106494969802211430E
:10426000044A516105E00349496980229143014AAA
:104270005161704700F801400146054A50698009C4
:1042800080018A06920E1043014A50617047000077
:1042900000F8014070B505460C46494840780128B1
:1042A0001CD10020FFF7C8FA012809D100F0FCF862
:1042B000012044490870002041498880487035E059
:1042C0002846FEF713F93E49488000F0CFF8032056
:1042D0003C49087000203A49487027E03848407847
:1042E00002281CD10020FFF7A7FA022809D100F00C
:1042F000DBF80220334908700020314948804870BB
:1043000014E02846FEF7F2F82D49888000F090F876
:1043100004202C49087000202949487006E02848EC
:104320004078042802D101202649487025480078A9
:10433000032815D122484088002805D100F0B4F8A0
:1043400005202049087004E01D484088401E1C4993
:1043500048801B488079012823D100F0A5F820E08F
:104360001848007804281CD115488088002805D1F9
:1043700000F09AF805201349087004E0104880887E
:10438000401E0F4988800E488079012809D100F02D
:104390008BF803200B4908702846FEF7A7F8084958
:1043A000488008480078032803D00648007804288D
:1043B00002D10121617101E00021617170BD000035
:1043C0003A000020B600002010B50024FDF776FA70
:1043D000012109031448FDF796FE01280AD10520A2
:1043E00000F0A0FE012109030F48FDF78CFE012813
:1043F00000D10124012C07D10C48807901280AD072
:1044000001200A49887106E008488079012802D114
:1044100000200649887105488079012802D10020D2
:10442000FFF70AFA10BD0000800C00403A0000209F
:1044300010B5FEF713FFFEF721FF012189020A489C
:10444000FDF76BFE012189020748FDF766FE012397
:104450001A4659020448FDF7A9FB01231A465902DE
:104460000148FDF7A3FB10BD000D004010B5FEF79D
:10447000F5FEFEF703FF012189020A48FDF74FFE12
:10448000012189020748FDF74AFE01231A46590215
:104490000448FDF78BFB01231A4659020148FDF73A
:1044A00085FB10BD000D004010B5FEF7D7FEFEF7EE
:1044B000F5FE0023012251020948FDF777FB002396
:1044C000012251020648FDF771FB012189020448CF
:1044D000FDF723FE012189020148FDF720FE10BDF2
:1044E000000D004010B50446012C02D0022C07D16B
:1044F00000E000BF0020FFF79FF90349087000E0CB
:1045000000BF00BF10BD0000B600002010B50022A3
:1045100080210248FEF70EFF10BD0000000C004095
:1045200010B50446A07801280DD1607900280AD181
:104530006078002807D1A0701A480078002802D1BE
:1045400001201849087017480078030000F07BF834
:104550000604050A0F14191E19E000F029F8114984
:10456000087014E000F022F80E4908700FE000F027
:104570002BF80C4908700AE000F028F80949087087
:1045800005E000F011F80749087000E000BF00BF27
:1045900004480078002802D10021E17001E00121E7
:1045A000E17010BD14020020002070470420704705
:1045B00010B5FFF7ABFF80210248FDF7B0FD0320E7
:1045C00010BD0000000C004004207047032070471D
:1045D0000FB410B503A9044B044A029800F050F838
:1045E00010BC08BC04B018477154000044020020FD
:1045F0000FB410B504A9074B02AA039800F040F8C5
:10460000044602A9002000F075FA204610BC08BC40
:1046100004B01847F54A00002021020C01D01021F7
:104620001046020A01D010460839020901D010468E
:10463000091F820801D01046891E420801D0881E39
:104640007047081A704730B47446641E2578641C9D
:10465000AB4204D3635D5B00E31830BC18471D46D2
:10466000F8E702E008C8121F08C1002AFAD1704713
:104670007047002001E001C1121F002AFBD17047E2
:10468000FFB591B00F460546002606E025280AD062
:10469000149A139990476D1C761C28780028F5D140
:1046A000304615B0F0BD002400940121F34A029475
:1046B00000E004436D1C2B780846203B98401042D4
:1046C000F7D128782A280ED00222287801463039DE
:1046D000092915D800990A23594330394018144341
:1046E0006D1C0090F1E701CF0090002805DA012051
:1046F00040030443009840420090022004436D1C94
:1047000028782E2815D10420044368786D1C2A28A7
:104710000AD101CF6D1C02900BE002990A2251438D
:10472000303940186D1C029028780146303909292B
:10473000F3D928786C2810D006DC4C281AD06828C9
:104740000ED06A2817D104E0742813D07A2812D129
:1047500010E00120400504430CE00121090501E0BF
:10476000032109050C436978814203D1012000052A
:1047700024186D1C6D1C28786E281ED00CDC632854
:1047800031D004DC00288BD0582811D1B2E0642845
:104790007BD069280CD178E073282DD004DC6F28F9
:1047A00070D0702804D1A7E075286CD078286BD021
:1047B000149A13999047761C62E06002400F022819
:1047C00007D003280AD0042838680AD006603F1DA5
:1047D00056E03868F11706604160F8E738680680EF
:1047E000F5E70670F3E738786946087400204874E6
:1047F00004A80390012003E0386803900020C04320
:104800003F1D61070FD5002101E00199491C029A63
:104810000191914213DA8142F7DB019A0399895C95
:104820000029F2D10BE0002101E00199491C01911E
:104830008142FADB019A0399895C0029F5D101993B
:104840000098139A401A00902146149B00F03CF9FE
:1048500001998019461807E0039803990078491CCC
:104860000391149A139990470198401E0190401C9F
:10487000F2D12146149B139A009800F015F986197D
:104880006D1C0AE741E033E034E00A200021049087
:1048900005916002410F022905D001CFC21794464D
:1048A000032905D007E0FF1DFF08FF0003CF06E046
:1048B00000B2C2179446042902D140B2C1178C46F7
:1048C00000226146944506DA0A46002140429141A1
:1048D0008C462D2102E0210504D52B216A46117654
:1048E000012103E0E10701D02021F7E7019155E024
:1048F0000A200BE0102009E0102004900021042081
:10490000044308200591029003E00820002105914E
:1049100004906002410F022905D001CF0022944685
:10492000032906D006E0FF1DFF08FF0003CF8C46D9
:1049300003E080B2042900D1C0B200210191210717
:104940002CD529780391702906D0049A1021059B53
:104950004A401A4305D00EE040216A4611760121F3
:1049600008E06146014306D030216A46117603997A
:10497000517602210191049A0821059B4A401A436D
:104980000CD16146014301D1610707D530216A4648
:104990001176012101910299491E02912978582925
:1049A00004D037A103910FA90F910DE039A1F9E7C8
:1049B0006146059B049AFBF7CDFB039B8C469B5CF1
:1049C0000F9A521E0F92137061460143F0D10F9857
:1049D00007A9081A20300390600704D501200004BD
:1049E0008443029801E0012002900399884201DD8E
:1049F000401A00E000204118029001980918009820
:104A0000401A0090E00306D42146149B139A0098A4
:104A100000F05AF886190020049008E006A9085C06
:104A2000149A139990470498401C761C049001999D
:104A30008842F3DBE0030CD52146149B139A0098BF
:104A400000F042F8861904E0149A30201399904738
:104A5000761C0299481E02900029F5DC08E00F98A8
:104A60000F990078491C0F91149A13999047761C5E
:104A70000399481E03900029F1DCFAE60928010099
:104A800030313233343536373839616263646566C4
:104A90000000000030313233343536373839414286
:104AA0004344454600000000F8B5044600251E4674
:104AB0001746880404D405E039462020B0476D1C11
:104AC000641EF9D52846F8BDFFB50446002581B01F
:104AD0001E46C80301D5302700E02027880404D5EE
:104AE00005E038460399B0476D1C641EF9D5284689
:104AF00005B0F0BD0A68531C0B60107070470000D1
:104B0000F0B585B00446002004902248808AA04277
:104B10001ED22049898A601AFBF70CFE00901E48BD
:104B200001680098FBF734FC01901C48016801986B
:104B3000FBF798FB0746FBF765FE05460022184B7E
:104B4000FBF709FD03910290FBF798FE04901DE02E
:104B50001049898A081BFBF7EDFD00900E4801689B
:104B60000098FBF715FC01900C4801680198FBF7D1
:104B7000CEFB0746FBF746FE05460022084BFBF737
:104B8000EAFC03910290FBF779FE0490049805B0CB
:104B9000F0BD000040FBFF1F280000202C0000207B
:104BA0000000E03FF0B587B00446002713490A2013
:104BB000085EFBF7C7FD05460022114BFBF742FDDF
:104BC000039102900D49098961430846FBF7CEFD28
:104BD000054600220B4BFBF735FD01910090039B2E
:104BE000029AFBF713FC05910490FBF7E7FD0746DB
:104BF000002F00DA0027384607B0F0BD80FAFF1F0B
:104C00000000594000408F4010B5002400BFFCF761
:104C100055F8012801D1002010BD2046641C401C1D
:104C20000028F4D10120F7E710B501208007FCF738
:104C300065FB0120FCF750FB01231A464021234865
:104C4000FCF7B4FF01231A46202120484030FCF72E
:104C5000ADFF01231A4619031C488030FCF7A6FF5C
:104C600001231A46402119484030FCF79FFF0123D9
:104C70001A46082115484038FCF798FF01231A46C8
:104C800019461248FCF792FF01231A46D9020F4831
:104C90008030FCF78BFF1E20002805DBC206D20EF9
:104CA000012191400A4A116000BF00211E20FEF739
:104CB00005FB1E20002806DBC206D20E0121914012
:104CC000034A803A116000BF10BD0000C00C0040D4
:104CD00080E100E010B5FEF7A1FDFEF747F8FEF712
:104CE0009DF8FEF7EBFC10BD10B5012401F02AF988
:104CF000002800D1002410BD10B500240C48FBF79B
:104D00008FFA0C49884206D200F091FB0849094805
:104D1000FBF790FA0124002C08D02A232922120242
:104D2000FF2101310248801F00F036FD10BD000058
:104D3000960200200116042410B5012401F020F988
:104D4000002800D1002410BDF0B50446002B0CD182
:104D500025460E46002005E02F783770761C6D1C26
:104D6000471CB8B29042F7DB0EE0012B0CD1A7181C
:104D70007D1E0E46002005E02F783770761C6D1ED4
:104D8000471CB8B29042F7DBF0BD0000F7B584B025
:104D9000074616463B480068039000253A480068DD
:104DA00002900020019039480078002822D038482D
:104DB000007800281ED13748826928466D1C800083
:104DC0003A5034484069441E33480068844211D345
:104DD00031480068314909684018A0420AD3102DB3
:104DE00008D20598854205D228466D1C80003C50AB
:104DF000012001902648007800280CD003988642B4
:104E000001D2039E07E0029903984018B04202D2F3
:104E10000299039846182DE03068041FE007C00F80
:104E2000002800D125E03068441E1B480068001DA2
:104E300084421DD318480068184909684018A042E8
:104E400016D3102D14D2201F00F0BCF900280FD06B
:104E5000059885420CD2022D06D10198002803D076
:104E60007868A04200D104E028466D1C80003C50C8
:104E700000BF361D029903984018B042CCD828468E
:104E800007B0F0BD200200202402002031020020E3
:104E900032020020D40C0020280200202C02002026
:104EA000F0B58FB00E4635462C4620224D4907A856
:104EB000FBF792F94C4807684C48006806904C484C
:104EC0000078002809D14B4A4BA14DA0FFF780FB89
:104ED00053A0FFF77DFB00BFFEE752480078002893
:104EE00009D0444A50A146A0FFF772FB4CA0FFF73F
:104EF0006FFB00BFFEE701204A4908704DA0FFF795
:104F000067FB47A0FFF764FB00F0D2F84A49C86A84
:104F1000FFF75EFB42A0FFF75BFB2035BD4203D3EA
:104F200006983818A84202D20120444908702A463F
:104F30003846069900F064F94048007800284BD1C3
:104F40003D49086BFFF744FB35A0FFF741FB3C49A7
:104F50002068086060684860A0688860E068C86091
:104F60002069086160694861A0698861E069C86179
:104F70000846C068324A0A999268099B01930292D6
:104F8000039104902E48406800902D48089B0268C9
:104F90002CA00799FFF71CFB21A0FFF719FB28485D
:104FA000C069274A0E9992690D9B01930292039161
:104FB000049023484069009021480C9B026921A07D
:104FC0000B99FFF705FB16A0FFF702FB28A0FFF7E0
:104FD000FFFA13A0FFF7FCFA284600F0F9FB0FB028
:104FE000F0BD0000486400002002002024020020E0
:104FF0003002002034640000696E69745F6F6B00DA
:105000002825732920686173206173736572742089
:105010006661696C65642061742025732E00000050
:105020000D0A000031020020216F6E5F6661756C11
:1050300074000000000000008863000032020020BD
:10504000D40C0020202025733A20253038782020E9
:1050500025733A2025303878202025733A202530D2
:105060003878202025733A20253038780000000059
:105070003D3D3D3D3D3D3D3D3D3D3D3D3D3D3D3D60
:105080003D3D3D3D3D3D3D3D3D3D3D3D3D3D3D3D50
:105090003D3D3D3D3D3D3D3D3D3D3D3D3D3D3D3D40
:1050A0003D3D3D3D3D3D3D3D3D3D3D3D3D3D0000AA
:1050B00010B50549054B064A48680649FFF788FAC6
:1050C00005A0FFF785FA10BD88630000240C0020BE
:1050D000040C0020E40B00200D0A000010B504466B
:1050E0000C480068C02188430A49086008460068E7
:1050F000C02108430749086007492046FBF700F82C
:1051000006490870084600787D21C90048430449D3
:10511000088010BD0024004040420F002200002003
:10512000240000200146114A12884A43104B5A615C
:1051300000229A611A46126901231A430C4B1A6124
:1051400000BF0B4A1069C207D20F002A04D0012207
:1051500012040240002AF4D0054A12695208520093
:10516000034B1A6100229A6170470000240000205E
:1051700000E000E00146114A12784A43104B5A61A0
:1051800000229A611A46126901231A430C4B1A61D4
:1051900000BF0B4A1069C207D20F002A04D00122B7
:1051A00012040240002AF4D0054A12695208520043
:1051B000034B1A6100229A61704700002200002010
:1051C00000E000E010B501460B884A881F20C002AD
:1051D00010401F24E402A04206D118400F242403EB
:1051E000A04201D1012010BDFF2000021040472441
:1051F0002402A04201D10120F5E70020F3E70000DE
:1052000070B505460E4614461D48007800281CD08F
:105210001C480078002808D01B4988692146FFF700
:10522000D7F91AA0FFF7D4F907E01749C869214652
:10523000FFF7CEF915A0FFF7CBF9AC4201D22C460F
:1052400003E0A819A04200D2AC190F490869FFF782
:10525000BFF90EA0FFF7BCF908E021460CA02268B8
:10526000FFF7B6F909A0FFF7B3F9241DA819A0426A
:10527000F3D80EA0FFF7ACF904A0FFF7A9F970BDB1
:105280003202002033020020886300000D0A000073
:105290002020616464723A20253038782020202054
:1052A000646174613A202530387800003D3D3D3D11
:1052B0003D3D3D3D3D3D3D3D3D3D3D3D3D3D3D3D1E
:1052C0003D3D3D3D3D3D3D3D3D3D3D3D3D3D3D3D0E
:1052D00000000000FFB5FFB0FFB085B007461C46D8
:1052E0000021FFA8C1600121890202A8FAF78DFF01
:1052F0000221019100264802844204DD00207FB093
:105300007FB009B0F0BD00261FE00121890202A88C
:10531000FAF77BFF2246FFA8416902A8FCF752F981
:10532000A21E02A902312D4800F008FF054668467A
:10533000407A01026846007A0918A94203D1012087
:10534000FFA9C86003E0701CC6B2022EDDDB00BFFF
:10535000FFA8C068012807D100232246394602A8C9
:10536000FFF7F2FC0120CAE700261FE001218902B5
:1053700002A8FAF74AFF2246FFA8816902A8FCF7B3
:1053800021F9A21E02A90231144800F0D7FE0546F9
:105390006846407A01026846007A0918A94203D19A
:1053A0000120FFA9C86003E0701CC6B2022EDDDB3D
:1053B00000BFFFA8C06801280DD10023224639464E
:1053C00002A8FFF7C1FC2246FFA8416902A8FCF72A
:1053D00031F9012093E7002091E70000FFFF000072
:1053E000F8B506460F4614461D46012000902A4691
:1053F0003946304600F01CF8002807D12A463946C5
:10540000304600F015F8002800D100902A462146C9
:10541000304600F00DF8002807D12A4621463046D4
:1054200000F006F8002800D100900098F8BD704701
:1054300070B5FFB0FFB082B005460E46144601209D
:105440008002844204DD00207FB07FB002B070BDD6
:10545000224631462846FCF7EDF82246314668469A
:10546000FCF7B0F822466946284600F09DFDEBE7C0
:1054700070B504460E46E5B229460548FEF702FE21
:1054800000BF0348FEF7DFFD0028FAD0284670BDB4
:105490000020014010B5002823D0124B0022001F2D
:1054A000196803E0814203D80A4649680029F9D106
:1054B000002A0AD01368841A9C4204D10068181884
:1054C0001060104602E0506000E01860002907D02C
:1054D00002680B1A934203D10B68D2180260496824
:1054E000416010BD4802002010B5FFF7F3FBFEF746
:1054F000C1FA10BD10B520211448FCF704FE0028A5
:1055000003D113480078401C00E0002010490870C7
:10551000012109030D484030FCF7F5FD002803D1B7
:105520000C480078401C00E000200A490870402127
:105530000648FCF7E8FD002803D107480078401C26
:1055400000E000200449087010BD0000000D00407C
:1055500036000020370000203800002010B5094830
:10556000C08800280ADD80210748FCF7CCFD002810
:1055700001D1FDF78DFCFDF779FC01E0FDF73AFC68
:1055800010BD000002000020C00C00401CB5FEF75A
:1055900089FCFFF7A9FF00F09FFC00F077FCFFF704
:1055A00043FBFDF761FA8FE0484800780128FAD103
:1055B000002046490870FDF757FA4548FDF734F8D2
:1055C00000281AD100BF434840794006C00F002888
:1055D00012D1414949794022914340313E4A5171AB
:1055E0004906C90F890140221140084639494979C5
:1055F00091430143374A517100BFFFF77BFFFFF72B
:10560000ADFF00F0E7FC3248017868460170304891
:105610004178684641702E488178684681702C48F0
:10562000C1786846C1702A480179684601712848E6
:105630004179684641712948019A009900F06EFB52
:10564000264800F03FFA2248017868460170204859
:105650004178684641701E488178684681701C48D0
:10566000C1786846C1701A480179684601711848C6
:105670004179684641710199009800F0CBFA1848C9
:10568000FCF750FD154800F073FD1448FEF748FF85
:1056900012480178684601701048417868464170A8
:1056A0000E488178684681700C48C1786846C170A0
:1056B0000A48017968460171084841796846417194
:1056C00001990098FEF79CFB6EE7000000000020A7
:1056D000300000205002002066020020120000204E
:1056E00044000020F0B50B30C108C900144F00265B
:1056F000144A0FE003688B420BD38B4205D95C1A26
:105700004318456830C3083B00E04368136002C09B
:1057100004E0021D10680028ECD13046002803D1B7
:105720003868002801D00020F0BD064A0648106005
:10573000064A121AD208D20044C001203860D7E7C6
:105740004C02002048020020840E0020801E002011
:10575000F8B504460E462078B04202D1607803289E
:1057600001D00020F8BDA578FA2D01DD0020F9E771
:10577000281D275C3902E81C205C081887B2EA1C47
:105780002146044800F0DAFCB84201D00020E9E7E5
:105790000120E7E7FFFF0000FFB581B004460F4698
:1057A0001D46AA1EA11C094800F0C8FC064626702A
:1057B000301260702B4639462046039AFFF710FEE0
:1057C000002801D105B0F0BD0120FBE7FFFF00007C
:1057D00070B592B006460025402102A8FAF715FDE3
:1057E0003246102102A8FFF7D1FA0546002410E046
:1057F000A10002AB5A58E1006118134BC81813A15D
:10580000FEF7F6FE2021E000201808300E4A115461
:10581000641CAC42ECD3002D0DD00B48E9006B1892
:105820000C4900900CA2086A0D49FEF7D1FE0DA0AC
:10583000FEF7CEFE06E00749486AFEF7C9FE09A05A
:10584000FEF7C6FE12B070BD440C00202530386C47
:1058500078000000886300002E6178660000000078
:10586000E40B00200D0A00000FB470B5469E459D64
:1058700040A8008A062804DA002070BC08BC04B0E6
:10588000184700210CE004A8405C002802D004A8BE
:10589000441807E0402901DD0020EEE7481C81B2F2
:1058A000FF29F0DD00BFFF210531681A8D4218D0B5
:1058B00008DCE81FFA3800280DD001280DD0022896
:1058C00021D10CE0FC2813D0FD2813D0FF38FD387F
:1058D000002818D110E00020CFE70020CDE70020FD
:1058E000CBE731462046489B479AFDF7D1FFC4E7F6
:1058F0000020C2E70020C0E731462046489B479A77
:10590000FBF754FFB9E70020B7E7000000B5FF2020
:10591000053000F09DF8034600200649C870087164
:1059200003204870887008460371012048710220E6
:1059300000BD00003402002010B50C48007900289A
:1059400004D00A480079401E0849087107480079C8
:10595000002808D10121FF20053000F0EDF80320D8
:105960000249887010BD00BFFCE70000340200202F
:1059700010B5FFB085B0002432488078012839D1B5
:105980000021304881703048017880A801722E488B
:10599000417880A841722C48817880A881722A4879
:1059A000C17880A8C1722848017980A8017326486F
:1059B000417980A841732448817980A881730722A6
:1059C00082A93FA8FAF708FC0120FF210531F42243
:1059D0003D913E901B49F0396846FAF7FDFBFF22E6
:1059E00005321A4941A8FAF7F7FB41A80FC8FFF79B
:1059F0003BFF0446012C10D11348407912498979A4
:105A0000884203DB00207FB005B010BD0E4840790E
:105A1000401C0D4948710220F5E70B488078401E74
:105A2000C0B209498870002809D108464078401E54
:105A3000C0B24870002800D1E5E70220E3E7032068
:105A4000E1E70000180E002034020020180D0020AD
:105A50000146FF220532881A91421ED008DCC81F79
:105A6000FA3800280DD001280FD0022826D110E0E6
:105A7000FC2816D0FD2818D0FF38FD3800281DD18D
:105A800017E001200E4A9071704701200C4A907176
:105A9000FAE701200A4A9071F6E70120084A90715E
:105AA000F2E70120064A9071EEE70120044A907166
:105AB000EAE70320024A90710120E5E76420E3E76A
:105AC0003402002010B50446207801280ED16079F8
:105AD00000280BD1E078002808D120701548007804
:105AE000002803D101201349087060701148007824
:105AF000002806D0012805D0022808D0032810D19C
:105B00000AE00FE0FFF702FF0A4908700AE0FFF71A
:105B100013FF0849087005E0FFF72AFF05490870E0
:105B200000E000BF00BF03480078002800D160708B
:105B300010BD00003402002070B505460C46FF2160
:105B40000531681A8D4215D008DCE81FFA380028A4
:105B50000DD001280CD0022835D10AE0FC2810D045
:105B6000FD280FD0FF38FD3800282CD10BE02BE0AA
:105B70002AE029E03122FF21F631204600F028F802
:105B800022E021E020E011484079012805D10422DB
:105B90006421204600F01CF814E00C4840790228EB
:105BA00006D10422FF213331204600F011F809E02C
:105BB00006484079032805D10422FF2147312046B9
:105BC00000F006F800E000BF00BF70BD3402002006
:105BD000FEB506460C461546684606700321417020
:105BE00021128170C4702912017145710622694623
:105BF000064800F0A3FA0746684687713912C1715A
:105C0000082269460248FEF728FAFEBDFFFF0000A1
:105C10000078014013B582B00020019038484078E8
:105C20008007C00F002805D03649487C097C040253
:105C30000C4304E03349C87B897B04020C4301AB6D
:105C4000224603990298FDF70BF8012801D12E494D
:105C500008706846007B002806D16846407B002813
:105C600002D10120294908706846C07A00280AD16B
:105C70006846007B002806D16846407B002802D198
:105C80000120234908706846807A01280ED16846B1
:105C9000C07A00280AD16846007B002806D16846F1
:105CA000407B002802D101201A490870164800786C
:105CB000012805D118484078002801D11249087000
:105CC00012480078012805D113484078002801D1F6
:105CD0000E4908700E480078012805D10E4840781A
:105CE000002801D10A4908700A480078012805D126
:105CF00009484078002801D1064908701FBD0000FE
:105D000050020020230100206F0000206C000020C2
:105D10006D0000206E0000201200002037B582B018
:105D20000546002001906846007C002806D16846A0
:105D3000407C002802D10420504908706846C07B8E
:105D400000280AD16846007C002806D16846407CBD
:105D5000002802D10420494908706846807B012848
:105D60000ED16846C07B00280AD16846007C002816
:105D700006D16846407C002802D104203F490870C3
:105D80003F4840788007C00F002805D03D49487C37
:105D9000097C04020C4304E03A49C87B897B040275
:105DA0000C4301AB224604990398FCF759FF0128E4
:105DB00002D104203149087030480078002804D00E
:105DC00000202E490870012028702E48807CC007D2
:105DD000C00F002823D000201CE00C2800DB1DE0B1
:105DE0006946CA7B430027491A31C95C8A420FD1F0
:105DF00069460A7C430023491A31591849788A4276
:105E000006D16946497C002902D101211E4A117040
:105E1000411C88B21B49497E8142DEDC00BF194823
:105E2000807C0221084002281CD115484078800758
:105E3000C00F002805D01348817D427D0C02144319
:105E400004E01048017DC27C0C0214430D4B173353
:105E5000224604990398FCF703FF012802D105208C
:105E60000949087008480078002804D00020064935
:105E700008700120A87005B030BD00001800002097
:105E80005002002023010020190000200EB5FDF76C
:105E90008BFF0E48FCF7C8FB00280FD10C48C079D7
:105EA0000B4989790A4A5279094B00920191029073
:105EB0001A79D97898780123FDF744FF05490879C4
:105EC000FEF710FBFDF770FA0EBD00003000002059
:105ED000080300209000002010B596B02C210BA8DC
:105EE000FAF793F92C216846FAF78FF901242A2250
:105EF00021020BA8FBF766FB0BA80230FAF790F91A
:105F00000F49884200D10FE02A2229210902684660
:105F1000FBF758FB00A80230FAF782F908498842DB
:105F200001D1012400E00024002C02D1FEF7DCFEA8
:105F300001E0FEF701FFFEF7DFFE16B010BD000026
:105F40000116042410B50C490C48FAF773F90A49F4
:105F5000091D0A48FAF76EF9202107480830FAF7B8
:105F600054F92A2329221202FF2101310248801EFE
:105F7000FFF712FC10BD000092020020011604245D
:105F800010B52A2329221202FF2101310548FFF70B
:105F9000A1F9002803D1FFF7D5FF002010BD012093
:105FA000FCE700009002002070B503460C4600217B
:105FB000002000BF07E05D5C665CB54201D00020B8
:105FC00003E04D1CA9B29142F5DB00BF914200D124
:105FD000012070BD70B552488078012871D15048B9
:105FE00000880C286DDD4F4800786828F6D14C48B1
:105FF0000088801E84B24B48005D0002494A611C43
:10600000515C0843054622464649474800F096F849
:10601000A84276D100230C2244494248FEF794FE60
:106020000220424948710321404881713D48807AED
:1060300000023C494989FF2212021140091208431B
:10604000384948810846407A52283BD006DC11285E
:106050000BD0122813D0422851D119E082284BD0FE
:1060600083284AD099284AD148E030492D48FEF784
:106070000DF82F4908702D48FEF752F840E0002037
:106080002C4908802A49087000212B48C18137E03B
:1060900027480078012813D12248017AC2790802E2
:1060A00010432449098888420AD120491D48FEF737
:1060B0003DF81E48FEF734F8E12109011E48C18170
:1060C0001EE01FE01A480078012813D11548017A14
:1060D000C279080210431749098888420AD1134936
:1060E0001048FEF723F81148FEF71AF8E1210901DC
:1060F0001148C18104E004E002E001E000E000BFDB
:1061000000BF00BF06488078012807D1002004495D
:106110008870084601880348FAF777F870BD0000D8
:10612000B0070020B0030020FFFF0000B3070020ED
:106130000E0200201202002002000020F0B50346EB
:1061400014461D12DEB208E00A78491C7240064867
:10615000805C684006460548855C2046641E002831
:10616000F2D128023043F0BD88610000886200004F
:1061700010B50446FEF728F90249C87D2146FEF70E
:1061800089F810BD7000002000C1814001C080412D
:1061900001C0804100C1814001C0804100C18140F7
:1061A00000C1814001C0804101C0804100C18140E7
:1061B00000C1814001C0804100C1814001C08041D7
:1061C00001C0804100C1814001C0804100C18140C7
:1061D00000C1814001C0804100C1814001C08041B7
:1061E00001C0804100C1814000C1814001C08041A7
:1061F00001C0804100C1814001C0804100C1814097
:1062000000C1814001C0804101C0804100C1814086
:1062100000C1814001C0804100C1814001C0804176
:1062200001C0804100C1814000C1814001C0804166
:1062300001C0804100C1814001C0804100C1814056
:1062400000C1814001C0804100C1814001C0804146
:1062500001C0804100C1814001C0804100C1814036
:1062600000C1814001C0804101C0804100C1814026
:1062700000C1814001C0804100C1814001C0804116
:1062800001C0804100C1814000C0C101C30302C2FE
:10629000C60607C705C5C404CC0C0DCD0FCFCE0E66
:1062A0000ACACB0BC90908C8D81819D91BDBDA1AD6
:1062B0001EDEDF1FDD1D1CDC14D4D515D71716D646
:1062C000D21213D311D1D010F03031F133F3F232B6
:1062D00036F6F737F53534F43CFCFD3DFF3F3EFE26
:1062E000FA3A3BFB39F9F83828E8E929EB2B2AEA96
:1062F000EE2E2FEF2DEDEC2CE42425E527E7E62606
:1063000022E2E323E12120E0A06061A163A3A26275
:1063100066A6A767A56564A46CACAD6DAF6F6EAEE5
:10632000AA6A6BAB69A9A86878B8B979BB7B7ABA55
:10633000BE7E7FBF7DBDBC7CB47475B577B7B676C5
:1063400072B2B373B17170B0509091519353529235
:1063500096565797559594549C5C5D9D5F9F9E5EA5
:106360005A9A9B5B99595898884849894B8B8A4A15
:106370004E8E8F4F8D4D4C8C448485458747468685
:1063800082424383418180402866000018650000F6
:106390009C6600008066000084640000AC6400001D
:1063A000286A0000446A000048650000B4660000E6
:1063B000E4650000C4650000D4640000506700007C
:1063C00098670000C8660000806800004868000008
:1063D000A8690000546900000069000028690000F5
:1063E000046A0000E069000078690000D0670000DE
:1063F0000066000028670000F8670000586600008B
:10640000606A0000DC680000746700000467000038
:1064100024680000B8680000A465000088650000DA
:10642000636D5F6261636B74726163655F617373F7
:1064300065727400636D5F6261636B747261636542
:106440005F6661756C740000686400006C64000035
:106450007064000074640000806400007C640000CC
:106460007864000014650000523020005231200092
:106470005232200052332000504320004C52200062
:10648000523132003D3D3D3D3D3D3D3D3D3D3D2098
:10649000CFDFB3CCB6D1D5BBD0C5CFA2203D3D3DDB
:1064A0003D3D3D3D3D3D3D3D000000003D3D3D3D10
:1064B0003D3D3D3D3D3D3D3D20D6F7B6D1D5BBD020
:1064C000C5CFA2203D3D3D3D3D3D3D3D3D3D3D3D9A
:1064D000000000003D3D3D3D3D3D3D3D3D3D3D3DE0
:1064E0003D3D3D3D3D3D3D3D3D3D3D3D3D20BCC4F3
:1064F000B4E6C6F7D0C5CFA2203D3D3D3D3D3D3D74
:106500003D3D3D3D3D3D3D3D3D3D3D3D3D3D3D3DBB
:106510003D3D000050535200B9CCBCFEC3FBB3C696
:10652000A3BA2573A3ACD3B2BCFEB0E6B1BEBAC564
:10653000A3BA2573A3ACC8EDBCFEB0E6B1BEBAC524
:10654000A3BA257300000000B2E9BFB4B8FCB6E0FE
:10655000BAAFCAFDB5F7D3C3D5BBD0C5CFA2A3ACE4
:10656000C7EBD4CBD0D0A3BA61646472326C696ECD
:1065700065202D652025732573202D61202D662033
:10658000252E2A7300000000B7A2C9FAD7DCCFDF9E
:10659000B4EDCEF3B5C4B5D8D6B7A3BA25303878A4
:1065A00000000000B7A2C9FAB4E6B4A2C6F7B9DC8D
:1065B000C0EDB4EDCEF3B5C4B5D8D6B7A3BA253087
:1065C00038780000D4DAD6D0B6CFBBF2C2E3BBFA3B
:1065D000BBB7BEB3CFC2B7A2C9FAB4EDCEF3D2EC0B
:1065E000B3A30000D4DACFDFB3CC28257329D6D0EB
:1065F000B7A2C9FAB4EDCEF3D2ECB3A30000000009
:10660000B7A2C9FAD3C3B7A8B4EDCEF3A3ACD4AD47
:10661000D2F2A3BACAD4CDBCC7D0BBBBB5BD204152
:10662000524D20D7B4CCAC00B4EDCEF3A3BACEDE3D
:10663000B7A8BBF1C8A1D6F7D5BBD0C5CFA2A3AC34
:10664000C7EBBCECB2E9D6F7D5BBB5C4CFE0B9D83F
:10665000C5E4D6C300000000B7A2C9FAD3C3B7A8E7
:10666000B4EDCEF3A3ACD4ADD2F2A3BAC6F3CDBC95
:10667000D6B4D0D0B7C7B6D4C6EBB7C3CECA000025
:10668000D4DAD6D0B6CFBBF2C2E3BBFABBB7BEB347
:10669000CFC2B7A2C9FAB6CFD1D40000D4DACFDFC7
:1066A000B3CC28257329D6D0B7A2C9FAB6CFD1D496
:1066B00000000000BBF1C8A1BAAFCAFDB5F7D3C353
:1066C000D5BBCAA7B0DC0000B7A2C9FAB4E6B4A231
:1066D000C6F7B9DCC0EDB4EDCEF3A3ACD4ADD2F2C5
:1066E000A3BAC6F3CDBCB4D3B2BBD4CAD0EDB7C342
:1066F000CECAB5C4C7F8D3F2B6C1A1A2D0B4CAFD00
:10670000BEDD0000B7A2C9FAB5F7CAD4B4EDCEF326
:10671000A3ACD4ADD2F2A3BACAFDBEDDBCE0B2E2F6
:10672000B5E3C6A5C5E40000B7A2C9FAD3C3B7A8AC
:10673000B4EDCEF3A3ACD4ADD2F2A3BACEDED0A7E3
:10674000B5C4D2ECB3A3B7B5BBD8C2EB0000000010
:10675000B7A2C9FAD3B2B4EDCEF3A3ACD4ADD2F2A2
:10676000A3BAC8A1D6D0B6CFCFF2C1BFCAB1B3F6D3
:10677000B4ED0000B7A2C9FAB5F7CAD4B4EDCEF3B0
:10678000A3ACD4ADD2F2A3BAD6B4D0D020424B50F1
:106790005420D6B8C1EE0000B7A2C9FAB4E6B4A23C
:1067A000C6F7B9DCC0EDB4EDCEF3A3ACD4ADD2F2F4
:1067B000A3BAC6F3CDBCB4D3B2BBD4CAD0EDB7C371
:1067C000CECAB5C4C7F8D3F2C8A1D6B8C1EE00008E
:1067D000B7A2C9FAD3C3B7A8B4EDCEF3A3ACD4AD76
:1067E000D2F2A3BAC6F3CDBCD6B4D0D0CEB4B6A83C
:1067F000D2E5D6B8C1EE0000B7A2C9FAD3C3B7A894
:10680000B4EDCEF3A3ACD4ADD2F2A3BAC6F3CDBCF3
:10681000D6B4D0D0D0ADB4A6C0EDC6F7D6B8C1EED0
:1068200000000000B7A2C9FAB5F7CAD4B4EDCEF3A0
:10683000A3ACD4ADD2F2A3BAB7A2C9FACFF2C1BF0A
:10684000B2B6BBF100000000B7A2C9FAB4E6B4A228
:10685000C6F7B9DCC0EDB4EDCEF3A3ACD4ADD2F243
:10686000A3BAC8EBD5BBCAB1C6F3CDBCB7C3CECAB9
:10687000B2BBB1BBD4CAD0EDB5C4C7F8D3F20000E7
:10688000B7A2C9FAB4E6B4A2C6F7B9DCC0EDB4ED5C
:10689000CEF3A3ACD4ADD2F2A3BAB3F6D5BBCAB192
:1068A000C6F3CDBCB7C3CECAB2BBB1BBD4CAD0ED60
:1068B000B5C4C7F8D3F20000B7A2C9FAB5F7CAD475
:1068C000B4EDCEF3A3ACD4ADD2F2A3BACDE2B2BF55
:1068D000B5F7CAD4C7EBC7F300000000B7A2C9FAE6
:1068E000B5F7CAD4B4EDCEF3A3ACD4ADD2F2A3BA0B
:1068F0004E56494320CDA3BBFAC7EBC7F3000000B7
:10690000B7A2C9FAD7DCCFDFB4EDCEF3A3ACD4ADD8
:10691000D2F2A3BABEABC8B7B5C4CAFDBEDDD7DCE0
:10692000CFDFB4EDCEF30000B7A2C9FAD7DCCFDFDA
:10693000B4EDCEF3A3ACD4ADD2F2A3BAB2BBBEAB2E
:10694000C8B7B5C4CAFDBEDDD7DCCFDFB4EDCEF32A
:1069500000000000B7A2C9FAD7DCCFDFB4EDCEF358
:10696000A3ACD4ADD2F2A3BAD6B8C1EED7DCCFDF98
:10697000B4EDCEF300000000B7A2C9FAD7DCCFDF38
:10698000B4EDCEF3A3ACD4ADD2F2A3BAB6E8D0D472
:10699000B1A3B4E6B8A1B5E3D7B4CCACCAB1B7A241
:1069A000C9FAB4EDCEF30000B7A2C9FAB4E6B4A2B6
:1069B000C6F7B9DCC0EDB4EDCEF3A3ACD4ADD2F2E2
:1069C000A3BAB6E8D0D4B1A3B4E6B8A1B5E3D7B4BE
:1069D000CCACCAB1B7A2C9FAB4EDCEF30000000046
:1069E000B7A2C9FAD7DCCFDFB4EDCEF3A3ACD4ADF8
:1069F000D2F2A3BAC8EBD5BBCAB1B7A2C9FAB4EDFB
:106A0000CEF30000B7A2C9FAD7DCCFDFB4EDCEF3E6
:106A1000A3ACD4ADD2F2A3BAB3F6D5BBCAB1B7A278
:106A2000C9FAB4EDCEF30000B4EDCEF3A3BACFDFD4
:106A3000B3CCD5BB282530387829B7A2C9FAD2E71C
:106A4000B3F60000B4EDCEF3A3BAD6F7D5BB282534
:106A500030387829B7A2C9FAD2E7B3F600000000AF
:106A6000B7A2C9FAD3C3B7A8B4EDCEF3A3ACD4ADE3
:106A7000D2F2A3BAC6F3CDBCD6B4D0D0B3FD203089
:106A800020B2D9D7F7000000A86A0000000000205B
:106A900050020000940A0000386B000050020020F1
:106AA000305C00007246000081321E021BB4259645
:106AB00032B8410611F0411801010A110114810296
:106AC0002564BA0741032802043B02043912321A32
:106AD0000386211A460216ECFFE7FF3C23E7FF1B63
:106AE000C844B119042B8C4204323C072A37323790
:106AF00032A866100D686852867597784D55ECDCA3
:106B00002559071A3C021501A0053C06160520016F
:106B10000520220A1278B80808070605040302DADD
:106B200001801AF48E021364920359AF1401020318
:086B30001903011F0311127A81
:04000005000000C136
:00000001FF
